:020000040000FA
:04080000F9EF0BF011
:1008100003B272EF05F0F2B490EF05F09EB098EFDE
:1008200005F09EB2A0EF05F0F2A81AEF04F0F2B2C4
:1008300021EF04F0F2B01FEF04F0A8EF0BF0F296F6
:10084000F290CD90F2929EA02BEF04F00101533F65
:100850002BEF04F0542BAEC1B2F1AFC1B3F1B0C174
:10086000B4F1B1C1B5F1AAC1AEF1ABC1AFF1ACC148
:10087000B0F1ADC1B1F1A6C1AAF1A7C1ABF1A8C158
:10088000ACF1A9C1ADF1A2C1A6F1A3C1A7F1A4C168
:10089000A8F1A5C1A9F19EC1A2F19FC1A3F1A0C178
:1008A000A4F1A1C1A5F19AC19EF19BC19FF19CC188
:1008B000A0F19DC1A1F196C19AF197C19BF198C198
:1008C0009CF199C19DF1CECF96F1CFCF97F153C155
:1008D00098F154C199F1CF6ACE6A0101536B546B00
:1008E0009E90CD800FBC0F8E0FBA7AEF04F00F8A66
:1008F000A8EF0BF00F8C0FBEB6EF04F096C19AF183
:1009000097C19BF198C19CF199C19DF19AC19EF14B
:100910009BC19FF19CC1A0F19DC1A1F19EC1A2F11B
:100920009FC1A3F1A0C1A4F1A1C1A5F1A2C1A6F1EB
:10093000A3C1A7F1A4C1A8F1A5C1A9F1A6C1AAF1BB
:10094000A7C1ABF1A8C1ACF1A9C1ADF1AAC1AEF18B
:10095000ABC1AFF1ACC1B0F1ADC1B1F1AEC1B2F15B
:10096000AFC1B3F1B0C1B4F1B1C1B5F101015E6B7A
:100970005F6B606B616B96515E2797515F23985157
:100980006023995161239A515E279B515F239C51AB
:1009900060239D5161239E515E279F515F23A0518B
:1009A0006023A1516123A2515E27A3515F23A4516B
:1009B0006023A5516123A6515E27A7515F23A8514B
:1009C0006023A9516123AA515E27AB515F23AC512B
:1009D0006023AD516123AE515E27AF515F23B0510B
:1009E0006023B1516123B2515E27B3515F23B451EB
:1009F0006023B5516123D8900101613360335F33C7
:100A00005E33D8900101613360335F335E33D89039
:100A10000101613360335F335E3300C10CF101C10A
:100A20000DF102C10EF103C10FF104C110F105C1B6
:100A300011F106C112F107C113F108C114F109C186
:100A400015F10AC116F10BC117F134C135F111B816
:100A500035EF05F00101620E046F010E056F000E07
:100A6000066F000E076F3EEF05F00101A70E046F41
:100A7000020E056F000E066F000E076F5EC100F1DB
:100A80005FC101F160C102F161C103F1A9EC36F06F
:100A900003BF04D019BE02D019A0108C11A056EFCC
:100AA00005F010BA56EF05F00F80108A0CC100F166
:100AB0000DC101F10EC102F10FC103F110C104F12A
:100AC00011C105F112C106F113C107F114C108F1FA
:100AD00015C109F116C10AF117C10BF135C134F185
:100AE000A8EF0BF00392ABB2AB98AB88030103EE17
:100AF00000F080517F0BE92604C0EFFF802B81516D
:100B0000805D700BD8A48B8200008051815D700BDA
:100B1000D8A48B9281518019D8B40790A8EF0BF01C
:100B2000F2940101453FA8EF0BF0462BA8EF0BF024
:100B30009E900101533FA8EF0BF0542BA8EF0BF050
:100B40009E9211B875EF08F0040066A1A8EF05F0B9
:100B50008BB4B2EF05F010ACB2EF05F08B84109CB3
:100B6000B3EF05F08B9407B405EF06F007B005EF7F
:100B700006F01EC620F61FC621F61CC61EF61DC6B0
:100B80001FF61AC61CF61BC61DF606C608F607C6D3
:100B900009F604C606F605C607F602C604F603C63D
:100BA00005F626C628F627C629F624C626F625C643
:100BB00027F622C624F623C625F60EC610F60FC663
:100BC00011F60CC60EF60DC60FF60AC60CF60BC6CD
:100BD0000DF62EC630F62FC631F62CC62EF62DC6D3
:100BE0002FF62AC62CF62BC62DF616C618F617C6F3
:100BF00019F614C616F615C617F612C614F613C65D
:100C000015F68AEC38F038EC38F0077C07AC20EFAA
:100C100006F0C274C2B41AEF06F0C3CFB7F5C4CF62
:100C2000B8F50501D890B833B733D890B833B73397
:100C300021EF06F0C3CF55F1C4CF56F121EF06F0F6
:100C4000C28207B48EEF06F047C14BF148C14CF1A8
:100C500049C14DF14AC14EF15EC162F15FC163F11C
:100C600060C164F161C165F196C1B6F197C1B7F198
:100C700098C1B8F199C1B9F19AC1BAF19BC1BBF160
:100C80009CC1BCF19DC1BDF19EC1BEF19FC1BFF130
:100C9000A0C1C0F1A1C1C1F1A2C1C2F1A3C1C3F100
:100CA000A4C1C4F1A5C1C5F1A6C1C6F1A7C1C7F1D0
:100CB000A8C1C8F1A9C1C9F1AAC1CAF1ABC1CBF1A0
:100CC000ACC1CCF1ADC1CDF1AEC1CEF1AFC1CFF170
:100CD000B0C1D0F1B1C1D1F1B2C1D2F1B3C1D3F140
:100CE000B4C1D4F1B5C1D5F1B7C5B9F5B8C5BAF538
:100CF000B9C5BBF5BAC5BCF5010155515B275651C5
:100D00005C23E86A5D230E2E8EEF06F05CC157F17E
:100D10005DC158F15B6B5C6B5D6B078E0201002F50
:100D2000A8EF0BF03C0E006F1A50E00BE00AE866EB
:100D3000128818BE02D018B4108E00C10CF101C187
:100D40000DF102C10EF103C10FF104C110F105C193
:100D500011F106C112F107C113F108C114F109C163
:100D600015F10AC116F10BC117F134C135F181AA91
:100D70006EEF07F030A03FEF07F005012F51000A9A
:100D8000D8B46EEF07F005012F51010AD8B4F8EF7F
:100D900006F005012F51020AD8B439EF07F005011A
:100DA0002F51030AD8B439EF07F005012F51040A77
:100DB000D8B439EF07F005012F51050AD8B439EF3F
:100DC00007F005012F51060AD8B439EF07F00501E5
:100DD0002F51070AD8B439EF07F005012F51320A15
:100DE000D8B4F6EF06F02F6B6EEF07F06EEF07F05A
:100DF0000501576703EF07F0586703EF07F05967DE
:100E000003EF07F05A6707EF07F06EEF07F05BC5D7
:100E100000F15CC501F15DC502F15EC503F10101A0
:100E2000010E046F000E056F000E066F000E076FB7
:100E3000A9EC36F000C15BF501C15CF502C15DF5BE
:100E400003C15EF500672CEF07F001672CEF07F098
:100E500002672CEF07F003676EEF07F057C55BF5ED
:100E600058C55CF559C55DF55AC55EF50F886EEF3E
:100E700007F0050130673FEF07F06EEF07F00FBE98
:100E800054EF07F010A059EF07F00101476750EF4A
:100E900007F0486750EF07F0496750EF07F04A67DF
:100EA00054EF07F059EF07F007AE59EF07F06BEF7B
:100EB00007F00501312F6EEF07F03C0E316F302F38
:100EC0006EEF07F00101000E626FE00E636FA50E7A
:100ED000646F010E656F0501306B0F880501666B4D
:100EE00037B774EF07F066810CC100F10DC101F155
:100EF0000EC102F10FC103F110C104F111C105F1DE
:100F000012C106F113C107F114C108F115C109F1AD
:100F100016C10AF117C10BF135C134F100C10CF152
:100F200001C10DF102C10EF103C10FF104C110F1B5
:100F300005C111F106C112F107C113F108C114F185
:100F400009C115F10AC116F10BC117F134C135F110
:100F500001018A67B3EF07F08B67B3EF07F08C6787
:100F6000B3EF07F08D67B7EF07F0E7EF07F08EC13B
:100F700000F18FC101F190C102F191C103F10101B2
:100F8000010E046F000E056F000E066F000E076F56
:100F9000A9EC36F000C18EF101C18FF102C190F1D0
:100FA00003C191F10067DCEF07F00167DCEF07F0A8
:100FB0000267DCEF07F00367E7EF07F08AC18EF105
:100FC0008BC18FF18CC190F18DC191F10F80D57ED5
:100FD000D5BE6DD0D6CF47F1D7CF48F145C149F145
:100FE000E86AE8CF4AF119BE02D019A0108C10901F
:100FF00047C100F148C101F149C102F14AC103F101
:1010000001010A0E046F000E056F000E066F000E40
:10101000076FA9EC36F003AF1080010154A71DEF54
:1010200008F00F9A0F9C0F9E0101000E5E6F600E7C
:101030005F6F3D0E606F080E616F010147BF2DEFBE
:1010400008F048672DEF08F049672DEF08F04A6770
:101050002DEF08F0F28852EF08F0F2985E6B5F6BAC
:10106000606B616B966B976B986B996B9A6B9B6BD4
:101070009C6B9D6B9E6B9F6BA06BA16BA26BA36B1C
:10108000A46BA56BA66BA76BA86BA96BAA6BAB6BCC
:10109000AC6BAD6BAE6BAF6BB06BB16BB26BB36B7C
:1010A000B46BB56BD76AD66A0101456B466B0CC150
:1010B00000F10DC101F10EC102F10FC103F110C128
:1010C00004F111C105F112C106F113C107F114C1F8
:1010D00008F115C109F116C10AF117C10BF135C1AB
:1010E00034F1A8EF0BF0A8EF0BF00201002FBFEFD7
:1010F0000AF0D59ED6CF47F1D7CF48F145C149F187
:10110000E86AE8CF4AF1D76AD66A0101456B466BB7
:10111000D58E1A50E00BE00AE866128818BE02D09D
:1011200018B4108E17AE1C8C00C10CF101C10DF16A
:1011300002C10EF103C10FF104C110F105C111F19B
:1011400006C112F107C113F108C114F109C115F16B
:101150000AC116F10BC117F134C135F10FA0109A75
:1011600011B8BEEF08F00101620E046F010E056FA9
:10117000000E066F000E076FC7EF08F00101A70E03
:10118000046F020E056F000E066F000E076F47C159
:1011900000F148C101F149C102F14AC103F1A9ECD2
:1011A00036F003BFDAEF08F019BE02D019A0108C98
:1011B00011B00F800CC100F10DC101F10EC102F19F
:1011C0000FC103F110C104F111C105F112C106F103
:1011D00013C107F114C108F115C109F116C10AF1D3
:1011E00017C10BF135C134F102013C0E006F00C193
:1011F0000CF101C10DF102C10EF103C10FF104C1E7
:1012000010F105C111F106C112F107C113F108C1B6
:1012100014F109C115F10AC116F10BC117F134C15E
:1012200035F181AAC8EF09F030A099EF09F0050166
:101230002F51000AD8B4C8EF09F005012F51010A57
:10124000D8B452EF09F005012F51020AD8B493EF38
:1012500009F005012F51030AD8B493EF09F00501F5
:101260002F51040AD8B493EF09F005012F51050A54
:10127000D8B493EF09F005012F51060AD8B493EFC3
:1012800009F005012F51070AD8B493EF09F00501C1
:101290002F51320AD8B450EF09F02F6BC8EF09F084
:1012A000C8EF09F0050157675DEF09F058675DEF7A
:1012B00009F059675DEF09F05A6761EF09F0C8EF6F
:1012C00009F05BC500F15CC501F15DC502F15EC5C9
:1012D00003F10101010E046F000E056F000E066F91
:1012E000000E076FA9EC36F000C15BF501C15CF59B
:1012F00002C15DF503C15EF5006786EF09F0016785
:1013000086EF09F0026786EF09F00367C8EF09F07E
:1013100057C55BF558C55CF559C55DF55AC55EF511
:101320000F88C8EF09F00501306799EF09F0C8EFA1
:1013300009F00FBEAEEF09F010A0B3EF09F0010104
:101340004767AAEF09F04867AAEF09F04967AAEFD3
:1013500009F04A67AEEF09F0B3EF09F007AEB3EF5B
:1013600009F0C5EF09F00501312FC8EF09F03C0E77
:10137000316F302FC8EF09F00101000E626FE00EEF
:10138000636FA50E646F010E656F0501306B0F88EA
:101390000501666B37B7CEEF09F066810CC100F12D
:1013A0000DC101F10EC102F10FC103F110C104F131
:1013B00011C105F112C106F113C107F114C108F101
:1013C00015C109F116C10AF117C10BF135C134F18C
:1013D00000C10CF101C10DF102C10EF103C10FF109
:1013E00004C110F105C111F106C112F107C113F1D9
:1013F00008C114F109C115F10AC116F10BC117F1A9
:1014000034C135F101018A670DEF0AF08B670DEFEA
:101410000AF08C670DEF0AF08D6711EF0AF041EFCB
:101420000AF08EC100F18FC101F190C102F191C1AA
:1014300003F10101010E046F000E056F000E066F2F
:10144000000E076FA9EC36F000C18EF101C18FF1DB
:1014500002C190F103C191F1006736EF0AF0016714
:1014600036EF0AF0026736EF0AF0036741EF0AF041
:101470008AC18EF18BC18FF18CC190F18DC191F138
:101480000F80109047C100F148C101F149C102F13C
:101490004AC103F101010A0E046F000E056F000E30
:1014A000066F000E076FA9EC36F003AF1080010144
:1014B00054A767EF0AF00F9A0F9C0F9E0101000ED0
:1014C0005E6F600E5F6F3D0E606F080E616F47C10B
:1014D00000F148C101F149C102F14AC103F1010122
:1014E000140E046F050E056F000E066F000E076FD9
:1014F000A9EC36F003AF80EF0AF0F288A5EF0AF00E
:10150000F2985E6B5F6B606B616B966B976B986B21
:10151000996B9A6B9B6B9C6B9D6B9E6B9F6BA06B8F
:10152000A16BA26BA36BA46BA56BA66BA76BA86B3F
:10153000A96BAA6BAB6BAC6BAD6BAE6BAF6BB06BEF
:10154000B16BB26BB36BB46BB56B0CC100F10DC179
:1015500001F10EC102F10FC103F110C104F111C17B
:1015600005F112C106F113C107F114C108F115C14B
:1015700009F116C10AF117C10BF135C134F10400AC
:101580008BB4CAEF0AF010ACCAEF0AF08B84109C3F
:10159000CBEF0AF08B9407B41DEF0BF007B01DEFF3
:1015A0000BF01EC620F61FC621F61CC61EF61DC671
:1015B0001FF61AC61CF61BC61DF606C608F607C699
:1015C00009F604C606F605C607F602C604F603C603
:1015D00005F626C628F627C629F624C626F625C609
:1015E00027F622C624F623C625F60EC610F60FC629
:1015F00011F60CC60EF60DC60FF60AC60CF60BC693
:101600000DF62EC630F62FC631F62CC62EF62DC698
:101610002FF62AC62CF62BC62DF616C618F617C6B8
:1016200019F614C616F615C617F612C614F613C622
:1016300015F68AEC38F038EC38F0077C07AC38EF58
:101640000BF0C274C2B432EF0BF0C3CFB7F5C4CF06
:10165000B8F50501D890B833B733D890B833B7335D
:1016600039EF0BF0C3CF55F1C4CF56F139EF0BF082
:10167000C28207B4A6EF0BF047C14BF148C14CF151
:1016800049C14DF14AC14EF15EC162F15FC163F1E2
:1016900060C164F161C165F196C1B6F197C1B7F15E
:1016A00098C1B8F199C1B9F19AC1BAF19BC1BBF126
:1016B0009CC1BCF19DC1BDF19EC1BEF19FC1BFF1F6
:1016C000A0C1C0F1A1C1C1F1A2C1C2F1A3C1C3F1C6
:1016D000A4C1C4F1A5C1C5F1A6C1C6F1A7C1C7F196
:1016E000A8C1C8F1A9C1C9F1AAC1CAF1ABC1CBF166
:1016F000ACC1CCF1ADC1CDF1AEC1CEF1AFC1CFF136
:10170000B0C1D0F1B1C1D1F1B2C1D2F1B3C1D3F105
:10171000B4C1D4F1B5C1D5F1B7C5B9F5B8C5BAF5FD
:10172000B9C5BBF5BAC5BCF5010155515B2756518A
:101730005C23E86A5D230E2EA6EF0BF05CC157F127
:101740005DC158F15B6B5C6B5D6B078EA8EF0BF0B6
:1017500002C0E0FF005001C0D8FF1000A6B2AEEFFB
:101760000BF00CC0A9FF0BC0A8FFA69EA69CA684E8
:10177000F29E550EA76EAA0EA76EA682F28EA694B2
:10178000A6B2C0EF0BF00C2A1200A96EA69EA69C72
:10179000A680A8500C2A120004012C0E826F4DEC7A
:1017A0000FF0A4EC37F00C50C5EC0BF0E8CF00F1D3
:1017B0000C50C5EC0BF0E8CF01F101AFE5EF0BF0F9
:1017C0000101FF0E026FFF0E036F47EC37F0296730
:1017D000F1EF0BF00401200E826F4DEC0FF0F6EFED
:1017E0000BF004012D0E826F4DEC0FF051EC35F033
:1017F0001200306A076A0F6A106A116A126A136A65
:101800000F010D0EC16E860EC06E030EC26E0F016B
:10181000680E896E130E926E080E8A6E8A6AF30E37
:10182000936E8B6A900E946EC80EC5EC0BF0E8CFE9
:10183000E8FF1098E8A0108810A805D00E0E226EC0
:101840008E0E236E04D00F0E226E8F0E236E42EC8E
:1018500039F0F18EF19EFC0EC5EC0BF0E8CF0BF0E9
:101860000BA011800BA211820BA411840BA811886C
:10187000C90EC5EC0BF0E8CF17F0CA0EC5EC0BF0A3
:10188000E8CF18F0CB0EC5EC0BF0E8CF19F0CC0E7A
:10189000C5EC0BF0E8CF1AF0CD0EC5EC0BF0E8CF9D
:1018A0002FF01C6A1D6A0E6A01015B6B5C6B5D6B3D
:1018B000576B586BF29A0101476B486B496B4A6B47
:1018C0004B6B4C6B4D6B4E6B4F6B506B516B526B4C
:1018D000456B466BD76AD66A0F01280ED56EF28A21
:1018E0009D90B00ECD6E01015E6B5F6B606B616BA6
:1018F000626B636B646B656B666B676B686B696B64
:10190000536B546BCF6ACE6A0F9A0F9C0F9E9D80CB
:10191000760ECA6E9D8202013C0E006FCC6A160ED6
:10192000C5EC0BF0E8CF00F1170EC5EC0BF0E8CFDB
:1019300001F1180EC5EC0BF0E8CF02F1190EC5EC61
:101940000BF0E8CF03F1010103AFC1EF0CF0A4EC01
:1019500037F0160E0C6E00C10BF0AEEC0BF0170E4C
:101960000C6E01C10BF0AEEC0BF0180E0C6E02C148
:101970000BF0AEEC0BF0190E0C6E03C10BF0AEECDD
:101980000BF000C18AF101C18BF102C18CF103C1DE
:101990008DF100C18EF101C18FF102C190F103C13F
:1019A00091F11A0EC5EC0BF0E8CF00F11B0EC5EC5F
:1019B0000BF0E8CF01F11C0EC5EC0BF0E8CF02F103
:1019C0001D0EC5EC0BF0E8CF03F1010103AF17EFDB
:1019D0000DF0A4EC37F01A0E0C6E00C10BF0AEEC5B
:1019E0000BF01B0E0C6E01C10BF0AEEC0BF01C0EDD
:1019F0000C6E02C10BF0AEEC0BF01D0E0C6E03C1B1
:101A00000BF0AEEC0BF01A0EC5EC0BF0E8CF00F1CA
:101A10001B0EC5EC0BF0E8CF01F11C0EC5EC0BF072
:101A2000E8CF02F11D0EC5EC0BF0E8CF03F100C1C9
:101A300092F101C193F102C194F103C195F1240E19
:101A4000AC6E900EAB6E240EAC6E080EB86E000E2F
:101A5000B06E1F0EAF6E0401806B816B0F01900E94
:101A6000AB6E0F019D8A0301806B816BC26B8B9201
:101A7000E6EC3DF0E6EC3DF0880EC5EC0BF0E8CF6F
:101A800000F1890EC5EC0BF0E8CF01F1010101AFC7
:101A900062EF0DF0A4EC37F0880E0C6E00C10BF075
:101AA000AEEC0BF0890E0C6E01C10BF0AEEC0BF03E
:101AB000880EC5EC0BF0E8CF00F1890EC5EC0BF0F9
:101AC000E8CF01F100C140F601C141F602C142F682
:101AD00003C143F640EC41F0C5EC3BF0200EC5ECF1
:101AE0000BF0E8CF2FF505012F51FF0AD8A480EFA6
:101AF0000DF02F6B200E0C6E2FC50BF0AEEC0BF023
:101B00000501010E306F3C0E316F250EC5EC0BF058
:101B1000E8CF00F1260EC5EC0BF0E8CF01F1270E5F
:101B2000C5EC0BF0E8CF02F1280EC5EC0BF0E8CFC6
:101B300003F1010103AFB7EF0DF0A4EC37F0250E70
:101B40000C6E00C10BF0AEEC0BF0260E0C6E01C15A
:101B50000BF0AEEC0BF0270E0C6E02C10BF0AEECEE
:101B60000BF0280E0C6E03C10BF0AEEC0BF000C1B5
:101B700057F501C158F502C159F503C15AF500C125
:101B80005BF501C15CF502C15DF503C15EF5290E8F
:101B9000C5EC0BF0E8CF5FF5050160515F5DD8A0A3
:101BA0005FC560F5210EC5EC0BF0E8CF00F1220E09
:101BB000C5EC0BF0E8CF01F1230EC5EC0BF0E8CF3C
:101BC00002F1240EC5EC0BF0E8CF03F1010103AFE5
:101BD00018EF0EF0A4EC37F0210E0C6E00C10BF0E4
:101BE000AEEC0BF0220E0C6E01C10BF0AEEC0BF064
:101BF000230E0C6E02C10BF0AEEC0BF0240E0C6E3B
:101C000003C10BF0AEEC0BF0210EC5EC0BF0E8CFEE
:101C100000F1220EC5EC0BF0E8CF01F1230EC5EC6C
:101C20000BF0E8CF02F1240EC5EC0BF0E8CF03F186
:101C300000C161F501C162F502C163F503C164F53C
:101C40000DEC3BF0F3EC39F04BEC39F030A089EFC0
:101C50000EF005012F51020A16E005012F51030A6B
:101C600019E005012F51040A24E005012F51050A4E
:101C70002BE005012F51060A39E005012F51070A13
:101C80003FE089EF0EF0602F86EF0EF05FC560F544
:101C900089EF0EF0B0C500F101010F0E0017010130
:101CA0000051000A36E001010051050A32E086EFDA
:101CB0000EF0B0C500F101010F0E00170101005137
:101CC000000A27E086EF0EF00501B051000A21E07E
:101CD0000501B051150A1DE00501B051300A19E0A7
:101CE0000501B051450A15E086EF0EF00501B0512F
:101CF000000A0FE00501B051300A0BE086EF0EF04C
:101D00000501B051000A05E086EF0EF081BA7FEFC1
:101D100041F0DCEC38F007900001F28EF28C12AE4C
:101D200003D012BC60EF20F007B0EAEF32F00FB042
:101D300082EF2CF010BE82EF2CF012B882EF2CF064
:101D40000FB81DEF26F00301805181197F0BD8B425
:101D5000EAEF32F013EE00F081517F0BE126812B88
:101D6000E7CFE8FFE00BD8B4EAEF32F023EE82F0E1
:101D7000C2513F0BD926E7CFDFFFC22BDF50780AD5
:101D8000D8A4EAEF32F007808EC100F18FC101F1D3
:101D900090C102F191C103F10101040E046F000E24
:101DA000056F000E066F000E076FA9EC36F000AF4E
:101DB000E3EF0EF00101030E8E6F000E8F6F000E29
:101DC000906F000E916F03018251720AD8B466EFD2
:101DD0002CF08251520AD8B466EF2CF08251750A69
:101DE000D8B466EF2CF08251630AD8B4A4EF2FF078
:101DF0008251690AD8B415EF29F082517A0AD8B411
:101E000028EF2AF08251490AD8B4B4EF28F0825161
:101E1000500AD8B4D2EF27F08251700AD8B415EF27
:101E200028F08251540AD8B440EF28F08251740A45
:101E3000D8B486EF28F08251410AD8B463EF10F08D
:101E400082514B0AD8B461EF0FF082516D0AD8B4B9
:101E500096EF14F082514D0AD8B4AFEF14F08251CE
:101E6000730AD8B496EF2BF08251530AD8B4FBEF23
:101E70002BF082514C0AD8B412EF1CF08251760A32
:101E8000D8B43EEF15F08251590AD8B4E7EF13F0F9
:101E900012AE01D0128CDBEF2FF0040114EE00F033
:101EA00080517F0BE12682C4E7FF802B12000401E2
:101EB0000D0E826F4DEC0FF00A0E826F4DEC0FF09D
:101EC000120004014B0E826F4DEC0FF004012C0E3A
:101ED000826F4DEC0FF081B802D02FB630D00301E5
:101EE0008351430AD8B4A6EF0FF003018351630A6C
:101EF000D8B4A8EF0FF003018351520AD8B4AAEF67
:101F00000FF003018351720AD8B4ACEF0FF0030154
:101F10008351470AD8B4AEEF0FF003018351670A2B
:101F2000D8B4B0EF0FF003018351540AD8B4B2EF24
:101F30000FF003018351740AD8B421EF10F00301AC
:101F40008351550AD8B4B4EF0FF082D02F807AD0E5
:101F50002F9078D02F8276D02F9274D02F8472D089
:101F60002F9470D02F866ED084C330F185C331F1A9
:101F700086C332F187C333F10101296BF2EC37F0EC
:101F800069EC37F000C104F101C105F102C106F1AD
:101F900003C107F1E5EC37F0200EF86EF76AF66A38
:101FA0000900F5CF2CF10900F5CF2DF10900F5CF8F
:101FB0002EF10900F5CF2FF10900F5CF30F109001E
:101FC000F5CF31F10900F5CF32F10900F5CF33F14A
:101FD0000101296BF2EC37F069EC37F0A9EC36F02F
:101FE0000067FAEF0FF00167FAEF0FF00267FAEF00
:101FF0000FF0036701D025D004014E0E826F4DEC27
:102000000FF004016F0E826F4DEC0FF004014D0EC6
:10201000826F4DEC0FF00401610E826F4DEC0FF0FA
:102020000401740E826F4DEC0FF00401630E826F99
:102030004DEC0FF00401680E826F4DEC0FF0D9EFFC
:102040002FF02F96CD0E0C6E2FC00BF0AEEC0BF0D8
:10205000CD0EC5EC0BF0E8CF2FF02FB006D0040169
:10206000630E826F4DEC0FF005D00401430E826FBA
:102070004DEC0FF02FB206D00401720E826F4DECC2
:102080000FF005D00401520E826F4DEC0FF02FB40B
:1020900006D00401670E826F4DEC0FF005D00401ED
:1020A000470E826F4DEC0FF02FB606D00401740E70
:1020B000826F4DEC0FF005D00401540E826F4DEC91
:1020C0000FF0D9EF2FF00401410E826F4DEC0FF0AD
:1020D00003018351310AD8B407EF13F00301835190
:1020E000320AD8B437EF12F003018351330AD8B45F
:1020F000C0EF11F003018351340AD8B4B0EF10F0EF
:1021000003018351350AD8B48DEF10F004013F0E5E
:10211000826F4DEC0FF0D9EF2FF004012C0E826F7F
:102120004DEC0FF003018451300AD8B4A0EF10F049
:1021300003018451310AD8B4A8EF10F0F9EF11F07F
:102140008B900401300E826F4DEC0FF0AEEF10F06B
:102150008B800401310E826F4DEC0FF0D9EF2FF020
:10216000CC0EC5EC0BF0E8CF0BF004012C0E826F07
:102170004DEC0FF003018451310AD8B4D4EF10F0C4
:1021800003018451300AD8B4D6EF10F00301845112
:102190004D0AD8B4E0EF10F003018451540AD8B4CA
:1021A000E7EF10F0FEEF10F08A8401D08A940BAEB6
:1021B00004D00BAC02D00BBA21D0E00E0B1218D019
:1021C0001F0E0B168539E844E00B0B1211D0E00E00
:1021D0000B16E5EC37F085C332F186C333F101010C
:1021E000296BF2EC37F069EC37F000511F0B0B1242
:1021F000CC0E0C6E0BC00BF0AEEC0BF00401340EE9
:10220000826F4DEC0FF004012C0E826F4DEC0FF03D
:10221000CC0EC5EC0BF0E8CF1AF08AB406D004015E
:10222000300E826F4DEC0FF005D00401310E826F3D
:102230004DEC0FF004012C0E826F4DEC0FF01A38AC
:10224000E840070BE8CF82F40401300E82274DEC02
:102250000FF004012C0E826F4DEC0FF0A4EC37F060
:102260001A501F0BE8CF00F147EC37F032C182F46F
:102270000401300E82274DEC0FF033C182F40401CB
:10228000300E82274DEC0FF004012C0E826F4DECC6
:102290000FF0A4EC37F02DC000F100AF0BD0FF0E13
:1022A000016FFF0E026FFF0E036F04012D0E826F90
:1022B0004DEC0FF047EC37F031C182F40401300EE1
:1022C00082274DEC0FF032C182F40401300E8227D8
:1022D0004DEC0FF033C182F40401300E82274DEC37
:1022E0000FF004012C0E826F4DEC0FF0A4EC37F0D0
:1022F0002CC000F147EC37F031C182F40401300EFC
:1023000082274DEC0FF032C182F40401300E822797
:102310004DEC0FF033C182F40401300E82274DECF6
:102320000FF004012C0E826F4DEC0FF0A4EC37F08F
:102330002EC000F100AF0BD0FF0E016FFF0E026F39
:10234000FF0E036F04012D0E826F4DEC0FF047EC72
:1023500037F031C182F40401300E82274DEC0FF0CA
:1023600032C182F40401300E82274DEC0FF033C1EC
:1023700082F40401300E82274DEC0FF0D9EF2FF0DC
:10238000CB0EC5EC0BF0E8CF0BF004012C0E826FE6
:102390004DEC0FF003018451450AD8B4E4EF11F07D
:1023A00003018451440AD8B4E7EF11F003018451CA
:1023B000300AD8B4EAEF11F003018451310AD8B4DD
:1023C000EEEF11F0F9EF11F00B9EF3EF11F00B8E21
:1023D000F3EF11F0FC0E0B16F3EF11F0FC0E0B16E1
:1023E0000B80F3EF11F0CB0E0C6E0BC00BF0AEECCC
:1023F0000BF00401330E826F4DEC0FF004012C0E34
:10240000826F4DEC0FF0CB0EC5EC0BF0E8CF19F05E
:1024100019BE12EF12F00401450E826F4DEC0FF061
:1024200017EF12F00401440E826F4DEC0FF004011F
:102430002C0E826F4DEC0FF00401300E826F4DECCC
:102440000FF004012C0E826F4DEC0FF019B030EF3D
:1024500012F00401300E826F4DEC0FF035EF12F0E8
:102460000401310E826F4DEC0FF0D9EF2FF0CA0E40
:10247000C5EC0BF0E8CF0BF004012C0E826F4DEC95
:102480000FF003018451450AD8B473EF12F0030131
:102490008451440AD8B476EF12F0030184514D0AF6
:1024A000D8B47FEF12F003018451410AD8B479EF18
:1024B00012F003018451460AD8B47CEF12F00301F4
:1024C0008451560AD8B487EF12F003018451500AA0
:1024D000D8B492EF12F003018451520AD8B495EFA8
:1024E00012F09EEF12F00B9E98EF12F00B8E98EF09
:1024F00012F00B9C98EF12F00B8C98EF12F0FC0E80
:102500000B1685C3E8FF030B0B1298EF12F0C70EF2
:102510000B1685C3E8FF070BE846E846E8460B12B2
:1025200098EF12F00B8498EF12F00B9498EF12F0E2
:10253000CA0E0C6E0BC00BF0AEEC0BF0CA0EC5EC65
:102540000BF0E8CF18F00401320E826F4DEC0FF063
:1025500004012C0E826F4DEC0FF018BEB7EF12F095
:102560000401450E826F4DEC0FF0BCEF12F0040138
:10257000440E826F4DEC0FF004012C0E826F4DEC77
:102580000FF018C0E8FF030BE8CF82F40401300E0F
:1025900082274DEC0FF004012C0E826F4DEC0FF0F2
:1025A00018BCDAEF12F00401410E826F4DEC0FF00F
:1025B000DFEF12F00401460E826F4DEC0FF00401C4
:1025C0002C0E826F4DEC0FF018C0E8FF380BE8427C
:1025D000E842E842E8CF82F40401300E82274DEC55
:1025E0000FF004012C0E826F4DEC0FF018B400EFC9
:1025F00013F00401520E826F4DEC0FF005EF13F053
:102600000401500E826F4DEC0FF0D9EF2FF0C90E80
:10261000C5EC0BF0E8CF0BF004012C0E826F4DECF3
:102620000FF003018451450AD8B425EF13F00301DC
:102630008451440AD8B428EF13F0030184514D0AA1
:10264000D8B42BEF13F039EF13F00B9E33EF13F0E8
:102650000B8E33EF13F0F80E0B1685C3E8FF070B54
:102660000B1233EF13F0C90E0C6E0BC00BF0AEEC77
:102670000BF00401310E826F4DEC0FF004012C0EB3
:10268000826F4DEC0FF0C90EC5EC0BF0E8CF17F0E0
:1026900017BE06D00401450E826F4DEC0FF005D039
:1026A0000401440E826F4DEC0FF004012C0E826F7A
:1026B0004DEC0FF017C0E8FF070BE8CF82F40401E0
:1026C000300E82274DEC0FF004012C0E826F4DEC82
:1026D0000FF00780A4EC37F028C0E8FF003B004370
:1026E0000043030B47EC37F033C182F40401300E92
:1026F00082274DEC0FF004012C0E826F4DEC0FF091
:10270000A4EC37F028C001F1019F019D29C000F120
:10271000010147EC37F02FC182F40401300E82270B
:102720004DEC0FF030C182F40401300E82274DECE5
:102730000FF031C182F40401300E82274DEC0FF00E
:1027400032C182F40401300E82274DEC0FF033C108
:1027500082F40401300E82274DEC0FF004012C0EA0
:10276000826F4DEC0FF0A4EC37F02AC001F12BC0C2
:1027700000F1D89001330033D890013300330101C8
:1027800047EC37F02FC182F40401300E82274DEC64
:102790000FF030C182F40401300E82274DEC0FF0AF
:1027A00031C182F40401300E82274DEC0FF032C1AA
:1027B00082F40401300E82274DEC0FF033C182F415
:1027C0000401300E82274DEC0FF0D9EF2FF0FC0EF4
:1027D000C5EC0BF0E8CF0BF003018351520AD8B4DB
:1027E0001EEF14F003018351720AD8B421EF14F0E4
:1027F00003018351500AD8B424EF14F0030183512C
:10280000700AD8B427EF14F003018351550AD8B4E5
:102810002AEF14F003018351750AD8B42DEF14F098
:1028200003018351430AD8B436EF14F003018351F6
:10283000630AD8B439EF14F042EF14F00B903CEF78
:1028400014F00B803CEF14F00B923CEF14F00B8271
:102850003CEF14F00B943CEF14F00B843CEF14F0BD
:102860000B963CEF14F00B863CEF14F00B983CEF0A
:1028700014F00B883CEF14F0FC0E0C6E0BC00BF048
:10288000AEEC0BF00401590E826F4DEC0FF011907D
:10289000119211941198FC0EC5EC0BF0E8CF0BF0DF
:1028A0000BA011800BA211820BA411840BA811881C
:1028B00011A062EF14F00401520E826F4DEC0FF084
:1028C00067EF14F00401720E826F4DEC0FF011A847
:1028D00071EF14F00401430E826F4DEC0FF076EFB0
:1028E00014F00401630E826F4DEC0FF011A280EF23
:1028F00014F00401500E826F4DEC0FF085EF14F0D0
:102900000401700E826F4DEC0FF011A48FEF14F0E4
:102910000401550E826F4DEC0FF094EF14F004019A
:10292000750E826F4DEC0FF0D9EF2FF004016D0E94
:10293000826F4DEC0FF003018351300AD8B4EEEFF3
:1029400014F003018351310AD8B401EF15F00301EB
:102950008351320AD8B414EF15F0DBEF2FF00401E5
:102960004D0E826F4DEC0FF0E5EC37F084C331F182
:1029700085C332F186C333F10101296BF2EC37F0E4
:1029800069EC37F003018351300AD8B4D6EF14F064
:1029900003018351310AD8B4DEEF14F003018351EF
:1029A000320AD8B4E6EF14F0DBEF2FF0FD0E0C6E18
:1029B00000C10BF0AEEC0BF0EEEF14F0FE0E0C6E5F
:1029C00000C10BF0AEEC0BF001EF15F0FF0E0C6E3A
:1029D00000C10BF0AEEC0BF014EF15F00401300E5B
:1029E000826F4DEC0FF004012C0E826F4DEC0FF056
:1029F000A4EC37F0FD0EC5EC0BF0E8CF00F125EFAD
:102A000015F00401310E826F4DEC0FF004012C0E15
:102A1000826F4DEC0FF0A4EC37F0FE0EC5EC0BF01E
:102A2000E8CF00F125EF15F00401320E826F4DEC76
:102A30000FF0A4EC37F004012C0E826F4DEC0FF078
:102A4000FF0EC5EC0BF0E8CF00F147EC37F031C1D9
:102A500082F40401300E82274DEC0FF032C182F473
:102A60000401300E82274DEC0FF033C182F40401D3
:102A7000300E82274DEC0FF0D9EF2FF00301835178
:102A8000300AD8B4E3EF16F003018351310AD8B409
:102A90001AEF17F003018351320AD8B4CFEF18F0C0
:102AA00003018351330AD8B484EF1AF00301835130
:102AB000340AD8B42AEF1BF003018351730AD8B447
:102AC000C5EF15F003018351760AD8B4C7EF15F0AE
:102AD00003018351740AD8B4B2EF15F00301835196
:102AE000540AD8B477EF15F0D8A4DBEF2FF0040127
:102AF000760E826F4DEC0FF00401540E826F4DEC98
:102B00000FF007840001880E0C6EE5EC37F0298188
:102B1000030184512D0AD8B490EF15F001012991D9
:102B200085C32FF186C330F187C331F188C332F1F9
:102B300089C333F1F2EC37F069EC37F000C10BF0E8
:102B4000AEEC0BF001C10BF0AEEC0BF0880EC5EC57
:102B50000BF0E8CF40F6890EC5EC0BF0E8CF41F65C
:102B6000BDEF15F00401760E826F4DEC0FF00401FD
:102B7000740E826F4DEC0FF007840001880E0C6E0E
:102B8000CCEC0BF007947FEF26F0C5EC15F00401B8
:102B9000760E826F4DEC0FF00401760E826F4DECD5
:102BA0000FF0078401EC34F004012C0E826F4DEC21
:102BB0000FF00101036B026B3BC601F13AC600F155
:102BC00001AFE8EF15F00101FF0E026FFF0E036F7A
:102BD00047EC37F02967EFEF15F0F4EF15F004013B
:102BE0002D0E826F4DEC0FF02FC182F40401300ED8
:102BF00082274DEC0FF030C182F40401300E8227A1
:102C00004DEC0FF031C182F40401300E82274DECFF
:102C10000FF032C182F40401300E82274DEC0FF028
:102C200033C182F40401300E82274DEC0FF0040111
:102C30002C0E826F4DEC0FF00101036B026B3DC651
:102C400001F13CC600F101AF2BEF16F00101FF0EC0
:102C5000026FFF0E036F47EC37F0296732EF16F073
:102C600037EF16F004012D0E826F4DEC0FF02FC1DF
:102C700082F40401300E82274DEC0FF030C182F453
:102C80000401300E82274DEC0FF031C182F40401B3
:102C9000300E82274DEC0FF032C182F40401300E69
:102CA00082274DEC0FF033C182F40401300E8227ED
:102CB0004DEC0FF004012C0E826F4DEC0FF0010172
:102CC000036B026B3FC601F13EC600F101AF6EEF30
:102CD00016F00101FF0E026FFF0E036F47EC37F095
:102CE000296775EF16F07AEF16F004012D0E826F4A
:102CF0004DEC0FF02FC182F40401300E82274DEC11
:102D00000FF030C182F40401300E82274DEC0FF039
:102D100031C182F40401300E82274DEC0FF032C134
:102D200082F40401300E82274DEC0FF033C182F49F
:102D30000401300E82274DEC0FF004012C0E826F3F
:102D40004DEC0FF00101036B026B37C601F136C683
:102D500000F101AFB1EF16F00101FF0E026FFF0E9F
:102D6000036F47EC37F02967B8EF16F0BDEF16F0A8
:102D700004012D0E826F4DEC0FF02FC182F404017F
:102D8000300E82274DEC0FF030C182F40401300E7A
:102D900082274DEC0FF031C182F40401300E8227FE
:102DA0004DEC0FF032C182F40401300E82274DEC5D
:102DB0000FF033C182F40401300E82274DEC0FF086
:102DC00007947FEF26F00401760E826F4DEC0FF032
:102DD0000401300E826F4DEC0FF004012C0E826F57
:102DE0004DEC0FF012EC38F0A4EC37F000C600F117
:102DF00001C601F147EC37F030C182F40401300E16
:102E000082274DEC0FF031C182F40401300E82278D
:102E10004DEC0FF032C182F40401300E82274DECEC
:102E20000FF033C182F40401300E82274DEC0FF015
:102E30007FEF26F00401760E826F4DEC0FF0040157
:102E4000310E826F4DEC0FF007840101036B026BB2
:102E500002C600F103C601F101AF33EF17F0FF0E18
:102E6000026FFF0E036F0101076B066B04C604F1CE
:102E700005C605F105AF41EF17F0FF0E066FFF0E17
:102E8000076FAEEC36F00101076B066B06C604F166
:102E900007C605F105AF51EF17F0FF0E066FFF0EE5
:102EA000076FAEEC36F00101076B066B08C604F144
:102EB00009C605F105AF61EF17F0FF0E066FFF0EB3
:102EC000076FAEEC36F0D8900101033302330133C3
:102ED0000033D8900101033302330133003304017E
:102EE0002C0E826F4DEC0FF00101036B026B01C1E0
:102EF00001F100C100F101AF83EF17F00101FF0EF6
:102F0000026FFF0E036F47EC37F029678AEF17F067
:102F10008FEF17F004012D0E826F4DEC0FF02FC1D3
:102F200082F40401300E82274DEC0FF030C182F4A0
:102F30000401300E82274DEC0FF031C182F4040100
:102F4000300E82274DEC0FF032C182F40401300EB6
:102F500082274DEC0FF033C182F40401300E82273A
:102F60004DEC0FF00101036B026B0AC600F10BC6BA
:102F700001F101AFC0EF17F0FF0E026FFF0E036FFC
:102F80000101076B066B0CC604F10DC605F105AF18
:102F9000CEEF17F0FF0E066FFF0E076FAEEC36F0A8
:102FA0000101076B066B0EC604F10FC605F105AFF4
:102FB000DEEF17F0FF0E066FFF0E076FAEEC36F078
:102FC0000101076B066B10C604F111C605F105AFD0
:102FD000EEEF17F0FF0E066FFF0E076FAEEC36F048
:102FE000D89001010333023301330033D89001013B
:102FF000033302330133003304012C0E826F4DEC96
:103000000FF00101036B026B01C101F100C100F17E
:1030100001AF10EF18F00101FF0E026FFF0E036FFA
:1030200047EC37F0296717EF18F01CEF18F0040190
:103030002D0E826F4DEC0FF02FC182F40401300E83
:1030400082274DEC0FF030C182F40401300E82274C
:103050004DEC0FF031C182F40401300E82274DECAB
:103060000FF032C182F40401300E82274DEC0FF0D4
:1030700033C182F40401300E82274DEC0FF00101C0
:10308000036B026B12C600F113C601F101AF4DEFE5
:1030900018F0FF0E026FFF0E036F0101076B066B46
:1030A00014C604F115C605F105AF5BEF18F0FF0E6D
:1030B000066FFF0E076FAEEC36F00101076B066B73
:1030C00016C604F117C605F105AF6BEF18F0FF0E39
:1030D000066FFF0E076FAEEC36F00101076B066B53
:1030E00018C604F119C605F105AF7BEF18F0FF0E05
:1030F000066FFF0E076FAEEC36F0D8900101033378
:10310000023301330033D89001010333023301331A
:10311000003304012C0E826F4DEC0FF00101036BA4
:10312000026B01C101F100C100F101AF9DEF18F088
:103130000101FF0E026FFF0E036F47EC37F02967A6
:10314000A4EF18F0A9EF18F004012D0E826F4DECDA
:103150000FF02FC182F40401300E82274DEC0FF0E6
:1031600030C182F40401300E82274DEC0FF031C1E2
:1031700082F40401300E82274DEC0FF032C182F44C
:103180000401300E82274DEC0FF033C182F40401AC
:10319000300E82274DEC0FF007947FEF26F00401EC
:1031A000760E826F4DEC0FF00401320E826F4DEC03
:1031B0000FF007840101036B026B1AC600F11BC6F6
:1031C00001F101AFE8EF18F0FF0E026FFF0E036F81
:1031D0000101076B066B1CC604F11DC605F105AFA6
:1031E000F6EF18F0FF0E066FFF0E076FAEEC36F02D
:1031F0000101076B066B1EC604F11FC605F105AF82
:1032000006EF19F0FF0E066FFF0E076FAEEC36F0FB
:103210000101076B066B20C604F121C605F105AF5D
:1032200016EF19F0FF0E066FFF0E076FAEEC36F0CB
:10323000D89001010333023301330033D8900101E8
:10324000033302330133003304012C0E826F4DEC43
:103250000FF00101036B026B01C101F100C100F12C
:1032600001AF38EF19F00101FF0E026FFF0E036F7F
:1032700047EC37F029673FEF19F044EF19F00401EC
:103280002D0E826F4DEC0FF02FC182F40401300E31
:1032900082274DEC0FF030C182F40401300E8227FA
:1032A0004DEC0FF031C182F40401300E82274DEC59
:1032B0000FF032C182F40401300E82274DEC0FF082
:1032C00033C182F40401300E82274DEC0FF001016E
:1032D000036B026B22C600F123C601F101AF75EF4B
:1032E00019F0FF0E026FFF0E036F0101076B066BF3
:1032F00024C604F125C605F105AF83EF19F0FF0ED2
:10330000066FFF0E076FAEEC36F00101076B066B20
:1033100026C604F127C605F105AF93EF19F0FF0E9D
:10332000066FFF0E076FAEEC36F00101076B066B00
:1033300028C604F129C605F105AFA3EF19F0FF0E69
:10334000066FFF0E076FAEEC36F0D8900101033325
:10335000023301330033D8900101033302330133C8
:10336000003304012C0E826F4DEC0FF00101036B52
:10337000026B01C101F100C100F101AFC5EF19F00D
:103380000101FF0E026FFF0E036F47EC37F0296754
:10339000CCEF19F0D1EF19F004012D0E826F4DEC36
:1033A0000FF02FC182F40401300E82274DEC0FF094
:1033B00030C182F40401300E82274DEC0FF031C190
:1033C00082F40401300E82274DEC0FF032C182F4FA
:1033D0000401300E82274DEC0FF033C182F404015A
:1033E000300E82274DEC0FF00101036B026B2AC6F1
:1033F00000F12BC601F101AF02EF1AF0FF0E026FD0
:10340000FF0E036F0101076B066B2CC604F12DC67E
:1034100005F105AF10EF1AF0FF0E066FFF0E076FF4
:10342000AEEC36F00101076B066B2EC604F12FC619
:1034300005F105AF20EF1AF0FF0E066FFF0E076FC4
:10344000AEEC36F00101076B066B30C604F131C6F5
:1034500005F105AF30EF1AF0FF0E066FFF0E076F94
:10346000AEEC36F0D8900101033302330133003360
:10347000D8900101033302330133003304012C0ED1
:10348000826F4DEC0FF00101036B026B01C101F182
:1034900000C100F101AF52EF1AF00101FF0E026FFF
:1034A000FF0E036F47EC37F0296759EF1AF05EEF14
:1034B0001AF004012D0E826F4DEC0FF02FC182F433
:1034C0000401300E82274DEC0FF030C182F404016C
:1034D000300E82274DEC0FF031C182F40401300E22
:1034E00082274DEC0FF032C182F40401300E8227A6
:1034F0004DEC0FF033C182F40401300E82274DEC05
:103500000FF007947FEF26F00401760E826F4DECEA
:103510000FF00401330E826F4DEC0FF004012C0EFE
:10352000826F4DEC0FF085C382F44DEC0FF0640E0A
:103530000D6E03018551320A02E16A0E0D6E030120
:103540008551330A02E1700E0D6E03018551340A74
:1035500002E1760E0D6E03018551350A02E17C0E03
:103560000D6E03018551360A02E1820E0D6E0301D4
:103570008651780A65E00DC00CF0E5EC37F0298142
:10358000030187512D0AD8B4C8EF1AF0010129911F
:1035900088C32FF189C330F18AC331F18BC332F173
:1035A0008CC333F1F2EC37F069EC37F000C10BF06B
:1035B000AEEC0BF001C10BF0AEEC0BF0E5EC37F02C
:1035C000298103018E512D0AD8B4E9EF1AF00101C7
:1035D00029918FC32FF190C330F191C331F192C380
:1035E00032F193C333F1F2EC37F069EC37F000C1FC
:1035F0000BF0AEEC0BF001C10BF0AEEC0BF0E5EC18
:1036000037F02981030195512D0AD8B40AEF1BF038
:103610000101299196C32FF197C330F198C331F17D
:1036200099C332F19AC333F1F2EC37F069EC37F019
:1036300000C10BF0AEEC0BF001C10BF0AEEC0BF0E7
:103640000DC00CF0CCEC0BF0CCEC0BF0CCEC0BF098
:103650007FEF26F00401760E826F4DEC0FF004012F
:10366000340E826F4DEC0FF003018451780AD8B408
:1036700002EF1CF03E0E0C6EE5EC37F029810301E1
:1036800085512D0AD8B447EF1BF00101299186C35B
:103690002FF187C330F188C331F189C332F18AC376
:1036A00033F1F2EC37F069EC37F000C10BF0AEEC1F
:1036B0000BF001C10BF0AEEC0BF0E5EC37F029811B
:1036C00003018C512D0AD8B468EF1BF00101299138
:1036D0008DC32FF18EC330F18FC331F190C332F11E
:1036E00091C333F1F2EC37F069EC37F000C10BF025
:1036F000AEEC0BF001C10BF0AEEC0BF0E5EC37F0EB
:103700002981030193512D0AD8B489EF1BF00101DF
:10371000299194C32FF195C330F196C331F197C32A
:1037200032F198C333F1F2EC37F069EC37F000C1B5
:103730000BF0AEEC0BF001C10BF0AEEC0BF0E5ECD6
:1037400037F0298103019A512D0AD8B4AAEF1BF052
:10375000010129919BC32FF19CC330F19DC331F12D
:103760009EC332F19FC333F1F2EC37F069EC37F0CE
:1037700000C10BF0AEEC0BF001C10BF0AEEC0BF0A6
:10378000E5EC37F029810301A1512D0AD8B4CBEF24
:103790001BF001012991A2C32FF1A3C330F1A4C3EF
:1037A00031F1A5C332F1A6C333F1F2EC37F069EC85
:1037B00037F000C10BF0AEEC0BF001C10BF0AEEC3A
:1037C0000BF0E5EC37F029810301A8512D0AD8B49C
:1037D000ECEF1BF001012991A9C32FF1AAC330F12D
:1037E000ABC331F1ACC332F1ADC333F1F2EC37F01E
:1037F00069EC37F000C10BF0AEEC0BF001C10BF03F
:10380000AEEC0BF03E0E0C6ECCEC0BF0CCEC0BF0F7
:10381000CCEC0BF0CCEC0BF0CCEC0BF0CCEC0BF0DC
:103820007FEF26F003018351300AD8B40DEF21F069
:1038300003018351310AD8B43AEF22F003018351D6
:10384000320AD8B4A8EF22F003018351330AD8B466
:10385000B8EF22F003018351340AD8B4C8EF22F044
:1038600003018351350AD8B423EF26F003018351B5
:10387000360AD8B451EF26F003018351370AD8B481
:10388000E5EF1EF003018351380AD8B483EF1FF02F
:1038900003018351460AD8B476EF25F00301835122
:1038A0004D0AD8B45EEF1DF0030183516D0AD8B400
:1038B00078EF1DF0030183515A0AD8B4B4EF21F018
:1038C00003018351490AD8B451EF27F00301835112
:1038D000500AD8B483EF26F003018351540AD8B4B8
:1038E000FCEF26F003018351630AD8B498EF1DF072
:1038F00003018351430AD8B490EF1EF003018351B2
:10390000730AD8B496EF1DF003018351610AD8B44D
:10391000ABEF1CF003018351650AD8B45DEF21F0D1
:1039200003018351450AD8B46BEF21F003018351A1
:10393000620AD8B479EF21F003018351420AD8B466
:1039400087EF21F003018351760AD8B495EF21F077
:10395000D8A4DBEF2FF004014C0E826F4DEC0FF07A
:103960000401610E826F4DEC0FF0F3EC39F00401AD
:103970002C0E826F4DEC0FF0A4EC37F0AFC500F1C8
:10398000010147EC37F031C182F40401300E822787
:103990004DEC0FF032C182F40401300E82274DEC61
:1039A0000FF033C182F40401300E82274DEC0FF08A
:1039B00004012C0E826F4DEC0FF0A4EC37F0B0C573
:1039C00000F1010147EC37F031C182F40401300EFF
:1039D00082274DEC0FF032C182F40401300E8227B1
:1039E0004DEC0FF033C182F40401300E82274DEC10
:1039F0000FF004012C0E826F4DEC0FF0A4EC37F0A9
:103A0000B1C500F1010147EC37F031C182F4040186
:103A1000300E82274DEC0FF032C182F40401300EDB
:103A200082274DEC0FF033C182F40401300E82275F
:103A30004DEC0FF004012C0E826F4DEC0FF0A4EC56
:103A400037F0B2C500F1010147EC37F031C182F423
:103A50000401300E82274DEC0FF032C182F40401D4
:103A6000300E82274DEC0FF033C182F40401300E8A
:103A700082274DEC0FF004012C0E826F4DEC0FF0FD
:103A8000A4EC37F0B6C500F1010147EC37F031C1C5
:103A900082F40401300E82274DEC0FF032C182F423
:103AA0000401300E82274DEC0FF033C182F4040183
:103AB000300E82274DEC0FF07FEF26F0E5EC37F06B
:103AC00084C333F1F2EC37F069EC37F0200E0C6E62
:103AD00000C10BF0AEEC0BF000C12FF505012F512A
:103AE000000A06E005012F51010A02E08DEC3AF0D0
:103AF00004014C0E826F4DEC0FF004014D0E826FED
:103B00004DEC0FF004012C0E826F4DEC0FF0A4EC85
:103B100037F02FC500F147EC37F033C182F40401D0
:103B2000300E82274DEC0FF07FEF26F07FEF41F053
:103B300004014C0E826F4DEC0FF00401630E826F96
:103B40004DEC0FF04BEC39F004012C0E826F4DEC74
:103B50000FF0ADEC1DF07FEF26F0A4EC37F0B5C50B
:103B600000F10101003B0F0E001747EC37F033C1A5
:103B700082F40401300E82274DEC0FF0B5C500F140
:103B800001010F0E0101001747EC37F033C182F439
:103B90000401300E82274DEC0FF004012D0E826FD0
:103BA0004DEC0FF0B4C500F10101003B0F0E001702
:103BB00047EC37F033C182F40401300E82274DEC1C
:103BC0000FF0B4C500F101010F0E0101001747EC21
:103BD00037F033C182F40401300E82274DEC0FF030
:103BE00004012D0E826F4DEC0FF0B3C500F1010101
:103BF000003B0F0E001747EC37F033C182F404018D
:103C0000300E82274DEC0FF0B3C500F101010F0E0D
:103C10000101001747EC37F033C182F40401300E84
:103C200082274DEC0FF00401200E826F4DEC0FF057
:103C3000B2C500F10F0E0101001747EC37F033C198
:103C400082F40401300E82274DEC0FF00401200EA7
:103C5000826F4DEC0FF0B1C500F101010101003B95
:103C60000F0E001747EC37F033C182F40401300E19
:103C700082274DEC0FF0B1C500F101010F0E0101DB
:103C8000001747EC37F033C182F40401300E82276D
:103C90004DEC0FF004013A0E826F4DEC0FF0B0C501
:103CA00000F10101003B0F0E001747EC37F033C164
:103CB00082F40401300E82274DEC0FF0B0C500F104
:103CC00001010F0E0101001747EC37F033C182F4F8
:103CD0000401300E82274DEC0FF004013A0E826F82
:103CE0004DEC0FF0AFC500F10101003B0F0E0017C6
:103CF00047EC37F033C182F40401300E82274DECDB
:103D00000FF0AFC500F101010F0E001747EC37F0BF
:103D100033C182F40401300E82274DEC0FF0120003
:103D200084C3E8FF0F0BE83AE8CFB5F585C3E8FF99
:103D30000F0B0501B51387C3E8FF0F0BE83AE8CF77
:103D4000B4F588C3E8FF0F0B0501B4138AC3E8FF7D
:103D50000F0BE83AE8CFB3F58BC3E8FF0F0B050173
:103D6000B3138DC3E8FF0F0BE8CFB2F58FC3E8FFA5
:103D70000F0BE83AE8CFB1F590C3E8FF0F0B050150
:103D8000B11392C3E8FF0F0BE83AE8CFB0F593C345
:103D9000E8FF0F0B0501B01395C3E8FF0F0BE83ADE
:103DA000E8CFAFF596C3E8FF0F0B0501AF13A6EC04
:103DB00039F004014C0E826F4DEC0FF00401430EFC
:103DC000826F4DEC0FF0A2EF1DF0078404014C0E42
:103DD000826F4DEC0FF00401370E826F4DEC0FF047
:103DE00004012C0E826F4DEC0FF005012E51130AC9
:103DF00006E005012E51170A0DE080EF1FF00101CA
:103E0000000E006F000E016F100E026F000E036FA8
:103E100013EF1FF00101000E006F000E016F000E86
:103E2000026F010E036F47EC37F02AC182F40401E0
:103E3000300E82274DEC0FF02BC182F40401300EBE
:103E400082274DEC0FF02CC182F40401300E822742
:103E50004DEC0FF02DC182F40401300E82274DECA1
:103E60000FF02EC182F40401300E82274DEC0FF0CA
:103E70002FC182F40401300E82274DEC0FF030C1C7
:103E800082F40401300E82274DEC0FF031C182F430
:103E90000401300E82274DEC0FF032C182F4040190
:103EA000300E82274DEC0FF033C182F40401300E46
:103EB00082274DEC0FF004012C0E826F4DEC0FF0B9
:103EC0000101200E006F000E016F000E026F000E48
:103ED000036F47EC37F031C182F40401300E8227C2
:103EE0004DEC0FF032C182F40401300E82274DEC0C
:103EF0000FF033C182F40401300E82274DEC0FF035
:103F000007947FEF26F00501216B226B236B246B56
:103F100004014C0E826F4DEC0FF00401380E826FDD
:103F20004DEC0FF004012C0E826F4DEC0FF00101EF
:103F3000200E006F000E016F000E026F000E036F67
:103F400047EC37F02AC182F40401300E82274DEC91
:103F50000FF02BC182F40401300E82274DEC0FF0DC
:103F60002CC182F40401300E82274DEC0FF02DC1DC
:103F700082F40401300E82274DEC0FF02EC182F442
:103F80000401300E82274DEC0FF02FC182F40401A2
:103F9000300E82274DEC0FF030C182F40401300E58
:103FA00082274DEC0FF031C182F40401300E8227DC
:103FB0004DEC0FF032C182F40401300E82274DEC3B
:103FC0000FF033C182F40401300E82274DEC0FF064
:103FD00004012C0E826F4DEC0FF025C500F126C5B3
:103FE00001F127C502F128C503F10101200E046F7C
:103FF000000E056F000E066F000E076FDAEC36F04C
:1040000000C133F501C134F502C135F503C136F500
:1040100047EC37F02AC182F40401300E82274DECC0
:104020000FF02BC182F40401300E82274DEC0FF00B
:104030002CC182F40401300E82274DEC0FF02DC10B
:1040400082F40401300E82274DEC0FF02EC182F471
:104050000401300E82274DEC0FF02FC182F40401D1
:10406000300E82274DEC0FF030C182F40401300E87
:1040700082274DEC0FF031C182F40401300E82270B
:104080004DEC0FF032C182F40401300E82274DEC6A
:104090000FF033C182F40401300E82274DEC0FF093
:1040A00057EC0FF0050133675DEF20F034675DEFEB
:1040B00020F035675DEF20F0366702D0FCEF20F08E
:1040C000129E129C21C500F122C501F123C502F107
:1040D00024C503F1899A400EC76E200EC66E9E96C7
:1040E000C69E0B0EC96EFF0E9EB602D0E82EFCD700
:1040F0009E96C69E02C1C9FFFF0E9EB602D0E82E54
:10410000FCD79E96C69E01C1C9FFFF0E9EB602D087
:10411000E82EFCD79E96C69E00C1C9FFFF0E9EB634
:1041200002D0E82EFCD79E96C69EC952FF0E9EB6C0
:1041300002D0E82EFCD70501200E326F040114EEE8
:1041400000F080517F0BE1269E96C69EC952FF0E5D
:104150009EB602D0E82EFCD7C9CFE7FF0401802B22
:104160000501322F9EEF20F0898A33C500F134C556
:1041700001F135C502F136C503F10101010E046FED
:10418000000E056F000E066F000E076FA9EC36F0EB
:1041900000C133F501C134F502C135F503C136F56F
:1041A00005013367DBEF20F03467DBEF20F0356784
:1041B000DBEF20F0366702D0FCEF20F021C500F1E4
:1041C00022C501F123C502F124C503F10101200E2E
:1041D000046F000E056F000E066F000E076FAEEC49
:1041E00036F000C121F501C122F502C123F503C15A
:1041F00024F5128EDBEF2FF00401450E826F4DEC9B
:104200000FF004014F0E826F4DEC0FF00401460ECB
:10421000826F4DEC0FF07FEF26F0078440EC41F009
:10422000A4EC37F02DC500F147EC37F004014C0E3B
:10423000826F4DEC0FF00401300E826F4DEC0FF0E9
:1042400004012C0E826F4DEC0FF031C182F4040199
:10425000300E82274DEC0FF032C182F40401300E93
:1042600082274DEC0FF033C182F40401300E822717
:104270004DEC0FF004012C0E826F4DEC0FF0A4EC0E
:1042800037F02EC500F147EC37F031C182F404015C
:10429000300E82274DEC0FF032C182F40401300E53
:1042A00082274DEC0FF033C182F40401300E8227D7
:1042B0004DEC0FF007947FEF26F004014C0E826F57
:1042C0004DEC0FF00401650E826F4DEC0FF069ECC0
:1042D0003BF07FEF26F004014C0E826F4DEC0FF0A7
:1042E0000401450E826F4DEC0FF080EC3BF07FEF48
:1042F00026F004014C0E826F4DEC0FF00401620EAB
:10430000826F4DEC0FF0AEEC3BF07FEF26F0040136
:104310004C0E826F4DEC0FF00401420E826F4DEC9B
:104320000FF097EC3BF07FEF26F004014C0E826F0C
:104330004DEC0FF00401760E826F4DEC0FF004018E
:104340002C0E826F4DEC0FF010A807D00401310E37
:10435000826F4DEC0FF07FEF26F00401300E826F7C
:104360004DEC0FF07FEF26F004014C0E826F4DEC08
:104370000FF004015A0E826F4DEC0FF004012C0E69
:10438000826F4DEC0FF040EC41F0A4EC37F00501EA
:104390002E51130A06E005012E51170A0DE0E5EF34
:1043A00021F00101000E006F000E016F100E026F70
:1043B000000E036FE5EF21F00101000E006F000E0B
:1043C000016F000E026F010E036F0101200E046FDA
:1043D000000E056F000E066F000E076FDAEC36F068
:1043E00047EC37F02AC182F40401300E82274DECED
:1043F0000FF02BC182F40401300E82274DEC0FF038
:104400002CC182F40401300E82274DEC0FF02DC137
:1044100082F40401300E82274DEC0FF02EC182F49D
:104420000401300E82274DEC0FF02FC182F40401FD
:10443000300E82274DEC0FF030C182F40401300EB3
:1044400082274DEC0FF031C182F40401300E822737
:104450004DEC0FF032C182F40401300E82274DEC96
:104460000FF033C182F40401300E82274DEC0FF0BF
:104470007FEF26F0078404014C0E826F4DEC0FF0A5
:104480000401310E826F4DEC0FF004012C0E826F8F
:104490004DEC0FF025C500F126C501F127C502F14D
:1044A00028C503F10101200E046F000E056F000EF8
:1044B000066F000E076FDAEC36F047EC37F02AC1D2
:1044C00082F40401300E82274DEC0FF02BC182F4F0
:1044D0000401300E82274DEC0FF02CC182F4040150
:1044E000300E82274DEC0FF02DC182F40401300E06
:1044F00082274DEC0FF02EC182F40401300E82278A
:104500004DEC0FF02FC182F40401300E82274DECE8
:104510000FF030C182F40401300E82274DEC0FF011
:1045200031C182F40401300E82274DEC0FF032C10C
:1045300082F40401300E82274DEC0FF033C182F477
:104540000401300E82274DEC0FF007947FEF26F028
:10455000078404014C0E826F4DEC0FF00401320E03
:10456000826F4DEC0FF09CEC3DF007947FEF26F04E
:10457000078404014C0E826F4DEC0FF00401330EE2
:10458000826F4DEC0FF0F9EC3DF0079445EF22F00F
:10459000078404014C0E826F4DEC0FF00401340EC1
:1045A000826F4DEC0FF004012C0E826F4DEC0FF07A
:1045B000E5EC37F084C32AF185C32BF186C32CF1D7
:1045C00087C32DF188C32EF189C32FF18AC330F13F
:1045D0008BC331F18CC332F18DC333F10101296BEF
:1045E000F2EC37F069EC37F0200E046F000E056F27
:1045F000000E066F000E076FBAEC36F000C121F511
:1046000001C122F502C123F503C124F5F3EC40F00A
:1046100038C5AFF539C5B0F53AC5B1F53BC5B2F50A
:104620003CC5B3F53DC5B4F53EC5B5F5ADEC1DF0E3
:1046300004012C0E826F4DEC0FF03FC500F140C518
:1046400001F141C502F142C503F10101000E046F01
:10465000000E056F010E066F000E076FDAEC36F0E4
:1046600047EC37F0296737EF23F03CEF23F00401E4
:104670002D0E826F4DEC0FF030C182F40401300E2C
:1046800082274DEC0FF031C182F40401300E8227F5
:104690004DEC0FF004012E0E826F4DEC0FF032C185
:1046A00082F40401300E82274DEC0FF033C182F406
:1046B0000401300E82274DEC0FF004012C0E826FA6
:1046C0004DEC0FF0A4EC37F043C500F144C501F107
:1046D00005EC31F004012C0E826F4DEC0FF0A4ECD0
:1046E00037F045C500F147EC37F031C182F40401E1
:1046F000300E82274DEC0FF032C182F40401300EEF
:1047000082274DEC0FF033C182F40401300E822772
:104710004DEC0FF004012C0E826F4DEC0FF00101F7
:10472000036B026B4CC501F14BC500F101AF9EEF6D
:1047300023F00101FF0E026FFF0E036F47EC37F00D
:104740002967A5EF23F0AAEF23F004012D0E826F55
:104750004DEC0FF02FC182F40401300E82274DEC96
:104760000FF030C182F40401300E82274DEC0FF0BF
:1047700031C182F40401300E82274DEC0FF032C1BA
:1047800082F40401300E82274DEC0FF033C182F425
:104790000401300E82274DEC0FF004012C0E826FC5
:1047A0004DEC0FF00101036B026B4EC501F14DC5DD
:1047B00000F101AFE1EF23F00101FF0E026FFF0EE8
:1047C000036F47EC37F02967E8EF23F0EDEF23F0B4
:1047D00004012D0E826F4DEC0FF02FC182F4040105
:1047E000300E82274DEC0FF030C182F40401300E00
:1047F00082274DEC0FF031C182F40401300E822784
:104800004DEC0FF032C182F40401300E82274DECE2
:104810000FF033C182F40401300E82274DEC0FF00B
:1048200004012C0E826F4DEC0FF00101036B026B43
:1048300050C501F14FC500F101AF24EF24F0010193
:10484000FF0E026FFF0E036F47EC37F029672BEF67
:1048500024F030EF24F004012D0E826F4DEC0FF0A8
:104860002FC182F40401300E82274DEC0FF030C1CD
:1048700082F40401300E82274DEC0FF031C182F436
:104880000401300E82274DEC0FF032C182F4040196
:10489000300E82274DEC0FF033C182F40401300E4C
:1048A00082274DEC0FF004012C0E826F4DEC0FF0BF
:1048B0000101036B026B52C501F151C500F101AF5B
:1048C00067EF24F00101FF0E026FFF0E036F47EC4C
:1048D00037F029676EEF24F073EF24F004012D0EFA
:1048E000826F4DEC0FF02FC182F40401300E82274D
:1048F0004DEC0FF030C182F40401300E82274DECF4
:104900000FF031C182F40401300E82274DEC0FF01C
:1049100032C182F40401300E82274DEC0FF033C116
:1049200082F40401300E82274DEC0FF004012C0EAE
:10493000826F4DEC0FF00101036B026B54C501F166
:1049400053C500F101AFAAEF24F00101FF0E026F81
:10495000FF0E036F47EC37F02967B1EF24F0B6EF95
:1049600024F004012D0E826F4DEC0FF02FC182F464
:104970000401300E82274DEC0FF030C182F40401A7
:10498000300E82274DEC0FF031C182F40401300E5D
:1049900082274DEC0FF032C182F40401300E8227E1
:1049A0004DEC0FF033C182F40401300E82274DEC40
:1049B0000FF004012C0E826F4DEC0FF00101036B20
:1049C000026B56C501F155C500F101AFEDEF24F0C2
:1049D0000101FF0E026FFF0E036F47EC37F02967EE
:1049E000F4EF24F0F9EF24F004012D0E826F4DEC6A
:1049F0000FF02FC182F40401300E82274DEC0FF02E
:104A000030C182F40401300E82274DEC0FF031C129
:104A100082F40401300E82274DEC0FF032C182F493
:104A20000401300E82274DEC0FF033C182F40401F3
:104A3000300E82274DEC0FF004012C0E826F4DECEE
:104A40000FF00101036B026B4AC501F149C500F18A
:104A500001AF30EF25F00101FF0E026FFF0E036F73
:104A600047EC37F0296737EF25F03CEF25F00401DC
:104A70002D0E826F4DEC0FF02FC182F40401300E29
:104A800082274DEC0FF030C182F40401300E8227F2
:104A90004DEC0FF031C182F40401300E82274DEC51
:104AA0000FF032C182F40401300E82274DEC0FF07A
:104AB00033C182F40401300E82274DEC0FF0040163
:104AC0002C0E826F4DEC0FF037C5E8FFE8B806D02A
:104AD0000401300E826F4DEC0FF005D00401310E51
:104AE000826F4DEC0FF007947FEF26F0E5EC37F086
:104AF00085C32AF186C32BF187C32CF188C32DF11E
:104B000089C32EF18AC32FF18BC330F18CC331F1ED
:104B10008DC332F18EC333F10101296BF2EC37F012
:104B200069EC37F00101010E046F000E056F000EF5
:104B3000066F000E076FA9EC36F0100E046F000E22
:104B4000056F000E066F000E076FBAEC36F000C15D
:104B500029F501C12AF502C12BF503C12CF523EC7F
:104B60003DF004014C0E826F4DEC0FF00401460E37
:104B7000826F4DEC0FF004012C0E826F4DEC0FF0A4
:104B800025C500F126C501F127C502F128C503F1AD
:104B90000101100E046F000E056F000E066F000E6F
:104BA000076FDAEC36F047EC37F02AC182F40401E3
:104BB000300E82274DEC0FF02BC182F40401300E31
:104BC00082274DEC0FF02CC182F40401300E8227B5
:104BD0004DEC0FF02DC182F40401300E82274DEC14
:104BE0000FF02EC182F40401300E82274DEC0FF03D
:104BF0002FC182F40401300E82274DEC0FF030C13A
:104C000082F40401300E82274DEC0FF031C182F4A2
:104C10000401300E82274DEC0FF032C182F4040102
:104C2000300E82274DEC0FF033C182F40401300EB8
:104C300082274DEC0FF07FEF26F00F98F9EC3DF056
:104C40003080DBEF2FF004014C0E826F4DEC0FF043
:104C50000401350E826F4DEC0FF004012C0E826FB3
:104C60004DEC0FF0A4EC37F00784B9C500F10794C0
:104C700047EC37F031C182F40401300E82274DEC4D
:104C80000FF032C182F40401300E82274DEC0FF098
:104C900033C182F40401300E82274DEC0FF07FEF18
:104CA00026F0BCEC3DF0A4EC37F037C500F147EC42
:104CB00037F004014C0E826F4DEC0FF00401360EFC
:104CC000826F4DEC0FF004012C0E826F4DEC0FF053
:104CD00031C182F40401300E82274DEC0FF032C155
:104CE00082F40401300E82274DEC0FF033C182F4C0
:104CF0000401300E82274DEC0FF07FEF26F057ECC9
:104D00000FF0DBEF2FF004014C0E826F4DEC0FF033
:104D10000401500E826F4DEC0FF004012C0E826FD7
:104D20004DEC0FF085C32AF186C32BF187C32CF11C
:104D300088C32DF189C32EF18AC32FF18BC330F1C3
:104D40008CC331F18DC332F18EC333F10101F2EC2A
:104D500037F069EC37F003018451530A0DE0030189
:104D600084514D0A38E00401780E826F4DEC0FF04B
:104D700057EC0FF0DBEF2FF00401530E826F4DEC78
:104D80000FF0250E0C6E00C10BF0AEEC0BF0260EF2
:104D90000C6E01C10BF0AEEC0BF0270E0C6E02C1D5
:104DA0000BF0AEEC0BF0280E0C6E03C10BF0AEEC6A
:104DB0000BF000C157F501C158F502C159F503C107
:104DC0005AF500C15BF501C15CF502C15DF503C197
:104DD0005EF560EF27F004014D0E826F4DEC0FF091
:104DE000290E0C6E00C10BF0AEEC0BF000C15FF5AC
:104DF00000C160F560EF27F004014C0E826F4DECAE
:104E00000FF00401540E826F4DEC0FF004012C0ED4
:104E1000826F4DEC0FF084C32AF185C32BF186C35A
:104E20002CF187C32DF188C32EF189C32FF18AC3DA
:104E300030F18BC331F18DC332F18EC333F10101F7
:104E4000F2EC37F069EC37F00101000E046F000E50
:104E5000056F010E066F000E076FBAEC36F0210EDB
:104E60000C6E00C10BF0AEEC0BF0220E0C6E01C10B
:104E70000BF0AEEC0BF0230E0C6E02C10BF0AEEC9F
:104E80000BF0240E0C6E03C10BF0AEEC0BF000C166
:104E900061F501C162F502C163F503C164F560EF1C
:104EA00027F004014C0E826F4DEC0FF00401490E07
:104EB000826F4DEC0FF004012C0E826F4DEC0FF061
:104EC000250EC5EC0BF0E8CF00F1260EC5EC0BF07B
:104ED000E8CF01F1270EC5EC0BF0E8CF02F1280E68
:104EE000C5EC0BF0E8CF03F147EC37F00AEC35F0F6
:104EF0000401730E826F4DEC0FF004012C0E826FD3
:104F00004DEC0FF0A4EC37F0290EC5EC0BF0E8CF18
:104F100000F147EC37F00AEC35F004016D0E826FBA
:104F20004DEC0FF004012C0E826F4DEC0FF05BC5C1
:104F300000F15CC501F15DC502F15EC503F147EC0E
:104F400037F00AEC35F00401730E826F4DEC0FF070
:104F500004012C0E826F4DEC0FF0A4EC37F060C50D
:104F600000F147EC37F00AEC35F004016D0E826F6A
:104F70004DEC0FF004012C0E826F4DEC0FF061C56B
:104F800000F162C501F163C502F164C503F1F6ECFD
:104F90002FF004012C0E826F4DEC0FF057EC0FF048
:104FA000DBEF2FF083C32AF184C32BF185C32CF1EF
:104FB00086C32DF187C32EF188C32FF189C330F149
:104FC0008AC331F18BC332F18CC333F10101F2ECAE
:104FD00037F069EC37F0160E0C6E00C10BF0AEEC3A
:104FE0000BF0170E0C6E01C10BF0AEEC0BF0180EAF
:104FF0000C6E02C10BF0AEEC0BF0190E0C6E03C17F
:105000000BF0AEEC0BF000C18AF101C18BF102C1D3
:105010008CF103C18DF100C18EF101C18FF102C18C
:1050200090F103C191F1B4EF28F083C32AF184C356
:105030002BF185C32CF186C32DF187C32EF188C3D4
:105040002FF189C330F18AC331F18BC332F18CC3A4
:1050500033F10101F2EC37F069EC37F000C18AF16D
:1050600001C18BF102C18CF103C18DF100C18EF140
:1050700001C18FF102C190F103C191F1B4EF28F0A9
:1050800083C32AF184C32BF185C32CF186C32DF190
:1050900087C32EF188C32FF189C330F18AC331F160
:1050A0008CC332F18DC333F10101F2EC37F069ECBE
:1050B00037F00101000E046F000E056F010E066F40
:1050C000000E076FBAEC36F01A0E0C6E00C10BF032
:1050D000AEEC0BF01B0E0C6E01C10BF0AEEC0BF046
:1050E0001C0E0C6E02C10BF0AEEC0BF01D0E0C6E24
:1050F00003C10BF0AEEC0BF000C192F101C193F1D2
:1051000002C194F103C195F1B4EF28F083C32AF1F1
:1051100084C32BF185C32CF186C32DF187C32EF1F7
:1051200088C32FF189C330F18AC331F18CC332F1C6
:105130008DC333F10101F2EC37F069EC37F0010176
:10514000000E046F000E056F010E066F000E076F54
:10515000BAEC36F000C192F101C193F102C194F1B1
:1051600003C195F1B4EF28F0160EC5EC0BF0E8CFB3
:1051700000F1170EC5EC0BF0E8CF01F1180EC5ECED
:105180000BF0E8CF02F1190EC5EC0BF0E8CF03F1FC
:1051900047EC37F00AEC35F00401730E826F4DECEA
:1051A0000FF004012C0E826F4DEC0FF08AC100F15C
:1051B0008BC101F18CC102F18DC103F147EC37F0D5
:1051C0000AEC35F00401730E826F4DEC0FF0040110
:1051D0002C0E826F4DEC0FF01A0EC5EC0BF0E8CFE1
:1051E00000F11B0EC5EC0BF0E8CF01F11C0EC5EC75
:1051F0000BF0E8CF02F11D0EC5EC0BF0E8CF03F188
:10520000F6EC2FF004012C0E826F4DEC0FF092C1E2
:1052100000F193C101F194C102F195C103F1F6ECE3
:105220002FF057EC0FF0DBEF2FF00401690E826FC7
:105230004DEC0FF004012C0E826F4DEC0FF00101CC
:10524000040E006F000E016F000E026F000E036F60
:1052500047EC37F02CC182F40401300E82274DEC6C
:105260000FF02DC182F40401300E82274DEC0FF0B7
:105270002EC182F40401300E82274DEC0FF02FC1B5
:1052800082F40401300E82274DEC0FF030C182F41D
:105290000401300E82274DEC0FF031C182F404017D
:1052A000300E82274DEC0FF032C182F40401300E33
:1052B00082274DEC0FF033C182F40401300E8227B7
:1052C0004DEC0FF004012C0E826F4DEC0FF001013C
:1052D0000B0E006F000E016F000E026F000E036FC9
:1052E00047EC37F02CC182F40401300E82274DECDC
:1052F0000FF02DC182F40401300E82274DEC0FF027
:105300002EC182F40401300E82274DEC0FF02FC124
:1053100082F40401300E82274DEC0FF030C182F48C
:105320000401300E82274DEC0FF031C182F40401EC
:10533000300E82274DEC0FF032C182F40401300EA2
:1053400082274DEC0FF033C182F40401300E822726
:105350004DEC0FF004012C0E826F4DEC0FF00101AB
:10536000370E006F000E016F000E026F000E036F0C
:1053700047EC37F02CC182F40401300E82274DEC4B
:105380000FF02DC182F40401300E82274DEC0FF096
:105390002EC182F40401300E82274DEC0FF02FC194
:1053A00082F40401300E82274DEC0FF030C182F4FC
:1053B0000401300E82274DEC0FF031C182F404015C
:1053C000300E82274DEC0FF032C182F40401300E12
:1053D00082274DEC0FF033C182F40401300E822796
:1053E0004DEC0FF004012C0E826F4DEC0FF0200EEF
:1053F000F86EF76AF66A04010900F5CF82F44DEC05
:105400000FF00900F5CF82F44DEC0FF00900F5CF55
:1054100082F44DEC0FF00900F5CF82F44DEC0FF063
:105420000900F5CF82F44DEC0FF00900F5CF82F4BE
:105430004DEC0FF00900F5CF82F44DEC0FF00900B0
:10544000F5CF82F44DEC0FF057EC0FF0DBEF2FF0BF
:105450008351630AD8A4D9EF2FF08451610AD8A4EC
:10546000D9EF2FF085516C0AD8A4D9EF2FF08651CF
:10547000410A3FE08651440A1BE08651420AD8B4F3
:105480008CEF2AF08651350AD8B465EF31F0865199
:10549000360AD8B4BAEF31F08651370AD8B423EFC0
:1054A00032F08651380AD8B481EF32F0D9EF2FF0BC
:1054B0000798079A04017A0E826F4DEC0FF00401F1
:1054C000780E826F4DEC0FF00401640E826F4DEC8C
:1054D0000FF00401550E826F4DEC0FF075EF2AF0BE
:1054E00004014C0E826F4DEC0FF057EC0FF0DBEF28
:1054F0002FF00788079A04017A0E826F4DEC0FF0A7
:105500000401410E826F4DEC0FF00401610E826FB9
:105510004DEC0FF069EF2AF00798078A04017A0E24
:10552000826F4DEC0FF00401420E826F4DEC0FF0D4
:105530000401610E826F4DEC0FF069EF2AF001015A
:105540006667AAEF2AF06767AAEF2AF06867AAEFF2
:105550002AF0696715D04F67B5EF2AF05067B5EFAD
:105560002AF05167B5EF2AF052670AD00101000E08
:10557000006F000E016F000E026F000E036F12002D
:1055800011B80AD00101620E046F010E056F000E02
:10559000066F000E076F09D00101A70E046F020EFF
:1055A000056F000E066F000E076F66C100F167C140
:1055B00001F168C102F169C103F1A9EC36F003BF42
:1055C00052EF2BF0119A119C0101000E046FA80EEE
:1055D000056F550E066F020E076F66C100F167C1B9
:1055E00001F168C102F169C103F166C186F167C1C9
:1055F00087F168C188F169C189F1A9EC36F003BF70
:105600000BD00101000E866FA80E876F550E886FB4
:10561000020E896F118A119C0E0EC5EC0BF0E8CFBB
:1056200018F10F0EC5EC0BF0E8CF19F1100EC5EC18
:105630000BF0E8CF1AF1110EC5EC0BF0E8CF1BF11F
:10564000F2EC35F086C104F187C105F188C106F19D
:1056500089C107F1A9EC36F00782B6EC35F0F2EC1F
:1056600035F00792B6EC35F086C100F187C101F143
:1056700088C102F189C103F10792B6EC35F0CC0E76
:10568000046FE00E056F870E066F050E076FA9EC1D
:1056900036F000C118F101C119F102C11AF103C1BC
:1056A0001BF13BD0119C119A0101800E006F1A0E64
:1056B000016F060E026F000E036F4FC104F150C15F
:1056C00005F151C106F152C107F1A9EC36F003AF63
:1056D00005D0A4EC37F0118C119A12000E0EC5EC17
:1056E0000BF0E8CF18F10F0EC5EC0BF0E8CF19F175
:1056F000100EC5EC0BF0E8CF1AF1110EC5EC0BF053
:10570000E8CF1BF14FC100F150C101F151C102F1CD
:1057100052C103F10782B6EC35F018C100F119C18E
:1057200001F11AC102F11BC103F112000401730E51
:10573000826F4DEC0FF004012C0E826F4DEC0FF0D8
:10574000078462C166F163C167F164C168F165C134
:1057500069F14BC14FF14CC150F14DC151F14EC1F6
:1057600052F157C159F158C15AF10794BCEC2BF0D2
:1057700057EC0FF0DBEF2FF066C100F167C101F1CC
:1057800068C102F169C103F1010147EC37F00AEC8D
:1057900035F00401630E826F4DEC0FF004012C0E06
:1057A000826F4DEC0FF04FC100F150C101F151C1BA
:1057B00002F152C103F1010147EC37F00AEC35F078
:1057C0000401660E826F4DEC0FF004012C0E826F07
:1057D0004DEC0FF0A4EC37F059C100F15AC101F1C2
:1057E000010147EC37F00AEC35F00401740E826FCA
:1057F0004DEC0FF0120010820401530E826F4DEC3D
:105800000FF004012C0E826F4DEC0FF083C32AF1D0
:1058100084C32BF185C32CF186C32DF187C32EF1F0
:1058200088C32FF189C330F18AC331F18BC332F1C0
:105830008CC333F10101F2EC37F069EC37F000C1B1
:1058400066F101C167F102C168F103C169F18EC35C
:105850002AF18FC32BF190C32CF191C32DF192C388
:105860002EF193C32FF194C330F195C331F196C358
:1058700032F197C333F10101F2EC37F069EC37F004
:1058800000C14FF101C150F102C151F103C152F108
:10589000E5EC37F099C32FF19AC330F19BC331F196
:1058A0009CC332F19DC333F10101F2EC37F069EC96
:1058B00037F000C159F101C15AF1BCEC2BF00401E1
:1058C0002C0E826F4DEC0FF076EF2CF0118E19A09C
:1058D00002D019AE108C18BE02D018A4108E03018D
:1058E0008251520A02E10F8201D00F928251750A51
:1058F00002E1108401D010948251550A02E1108611
:1059000001D0109611A003D011A401D010840784F7
:1059100010B2E4EF2CF010A4D0EF2CF0B6C166F179
:10592000B7C167F1B8C168F1B9C169F1BAC16AF12B
:10593000BBC16BF1BCC16CF1BDC16DF1BEC16EF1FB
:10594000BFC16FF1C0C170F1C1C171F1C2C172F1CB
:10595000C3C173F1C4C174F1C5C175F1C6C176F19B
:10596000C7C177F1C8C178F1C9C179F1CAC17AF16B
:10597000CBC17BF1CCC17CF1CDC17DF1CEC17EF13B
:10598000CFC17FF1D0C180F1D1C181F1D2C182F10B
:10599000D3C183F1D4C184F1D5C185F1D8EF2CF006
:1059A00062C166F163C167F164C168F165C169F103
:1059B0004BC14FF14CC150F14DC151F14EC152F1AB
:1059C00057C159F158C15AF107940FA006EF2DF0B5
:1059D00001019267F3EF2CF09367F3EF2CF09467DB
:1059E000F3EF2CF09567F7EF2CF006EF2DF09FEC1E
:1059F0002AF092C104F193C105F194C106F195C159
:105A000007F1A9EC36F003BFA1EF2FF09FEC2AF0CD
:105A10000101000E046F000E056F010E066F000EEF
:105A2000076FDAEC36F011A02AD011A228D047EC8B
:105A300037F0296701D005D004012D0E826F4DEC9F
:105A40000FF030C182F40401300E82274DEC0FF0CC
:105A500031C182F40401300E82274DEC0FF032C1C7
:105A600082F40401300E82274DEC0FF033C182F432
:105A70000401300E82274DEC0FF057EC0FF012A806
:105A8000C3D012981AC01BF01B3A1B42070E1B16FC
:105A900000011B50000AD8B4D2EF2DF000011B50BA
:105AA000010AD8B45EEF2DF000011B50020AD8B4F1
:105AB0005CEF2DF004EF2EF004EF2EF0A4EC37F0A5
:105AC0002AC001F12BC000F1D89001330033D890E7
:105AD000013300330101630E046F000E056F000EE9
:105AE000066F000E076FDAEC36F0280E046F000E1A
:105AF000056F000E066F000E076FA9EC36F000C1AF
:105B00002DF0A4EC37F028C001F1019F019D29C0C0
:105B100000F10101A40E046F000E056F000E066F68
:105B2000000E076FDAEC36F000C12CF000C104F172
:105B300001C105F102C106F103C107F1640E006F56
:105B4000000E016F000E026F000E036FA9EC36F01D
:105B5000050E046F000E056F000E066F000E076F36
:105B6000DAEC36F000C104F101C105F102C106F121
:105B700003C107F1A4EC37F02DC000F1A9EC36F019
:105B800000C12EF02EC0E8FF050F2D5C03E78A84CC
:105B900004EF2EF02EC0E8FF0A0F2D5C01E68A9478
:105BA00004EF2EF000C124F101C125F102C126F15C
:105BB00003C127F1A4EC37F0AAEC37F01A501F0B01
:105BC000E8CF00F10101640E046F000E056F000EB6
:105BD000066F000E076FBAEC36F024C104F125C140
:105BE00005F126C106F127C107F1A9EC36F003BF84
:105BF00002D08A9401D08A8424C100F125C101F128
:105C000026C102F127C103F100C124F101C125F130
:105C100002C126F103C127F110AE4DD0109E00C184
:105C200008F101C109F102C10AF103C10BF147EC0E
:105C300037F030C1D6F131C1D7F132C1D8F133C11B
:105C4000D9F108C100F109C101F10AC102F10BC18A
:105C500003F101016C0E046F070E056F000E066F55
:105C6000000E076FA9EC36F003BF04D00101550EFA
:105C7000DA6F1CD008C100F109C101F10AC102F1BB
:105C80000BC103F10101A40E046F060E056F000E97
:105C9000066F000E076FA9EC36F003BF04D00101B8
:105CA0007F0EDA6F03D00101FF0EDA6F1C8E11AE8A
:105CB000A1EF2FF0119E24C100F125C101F126C1F1
:105CC00002F127C103F111A005D011A203D00FB03A
:105CD000A1EF2FF010A474EF2EF00401750E826F67
:105CE0004DEC0FF079EF2EF00401720E826F4DEC47
:105CF0000FF004012C0E826F4DEC0FF047EC37F0E3
:105D0000296788EF2EF00401200E826F8BEF2EF0B2
:105D100004012D0E826F4DEC0FF030C182F40401AE
:105D2000300E82274DEC0FF031C182F40401300EA9
:105D300082274DEC0FF004012E0E826F4DEC0FF018
:105D400032C182F40401300E82274DEC0FF033C1D2
:105D500082F40401300E82274DEC0FF004016D0E29
:105D6000826F4DEC0FF004012C0E826F4DEC0FF0A2
:105D70004FC100F150C101F151C102F152C103F113
:105D8000010147EC37F00AEC35F00401480E826F50
:105D90004DEC0FF004017A0E826F4DEC0FF0040110
:105DA0002C0E826F4DEC0FF066C100F167C101F15E
:105DB00068C102F169C103F1010147EC37F00AEC57
:105DC00035F00401630E826F4DEC0FF004012C0ED0
:105DD000826F4DEC0FF066C100F167C101F168C13F
:105DE00002F169C103F101010A0E046F000E056F93
:105DF000000E066F000E076FBAEC36F0000E046F4F
:105E0000120E056F000E066F000E076FDAEC36F00B
:105E100047EC37F02AC182F40401300E82274DECA2
:105E20000FF02BC182F40401300E82274DEC0FF0ED
:105E30002CC182F40401300E82274DEC0FF02DC1ED
:105E400082F40401300E82274DEC0FF02EC182F453
:105E50000401300E82274DEC0FF02FC182F40401B3
:105E6000300E82274DEC0FF030C182F40401300E69
:105E700082274DEC0FF004012E0E826F4DEC0FF0D7
:105E800031C182F40401300E82274DEC0FF032C193
:105E900082F40401300E82274DEC0FF033C182F4FE
:105EA0000401300E82274DEC0FF00401730E826F57
:105EB0004DEC0FF004012C0E826F4DEC0FF0A4ECB2
:105EC00037F059C100F15AC101F105EC31F00FB2C0
:105ED0006DEF2FF00FA09FEF2FF004012C0E826FBB
:105EE0004DEC0FF0200EF86EF76AF66A0401090017
:105EF000F5CF82F44DEC0FF00900F5CF82F44DECB4
:105F00000FF00900F5CF82F44DEC0FF00900F5CF4A
:105F100082F44DEC0FF00900F5CF82F44DEC0FF058
:105F20000900F5CF82F44DEC0FF00900F5CF82F4B3
:105F30004DEC0FF00900F5CF82F44DEC0FF057EC6B
:105F40000FF00F90DBEF2FF00401630E826F4DEC2A
:105F50000FF004012C0E826F4DEC0FF0E1EC2FF0EE
:105F600004012C0E826F4DEC0FF054EC30F0040164
:105F70002C0E826F4DEC0FF0D0EC30F004012C0EA3
:105F8000826F4DEC0FF00101F80E006FCD0E016F26
:105F9000660E026F030E036FF6EC2FF004012C0E59
:105FA000826F4DEC0FF0E6EC30F057EC0FF0DBEFCA
:105FB0002FF057EC0FF00301C26B07901092EAEF3D
:105FC00032F0D8900E0EC5EC0BF0E8CF00F10F0EBA
:105FD000C5EC0BF0E8CF01F1100EC5EC0BF0E8CFEB
:105FE00002F1110EC5EC0BF0E8CF03F10101000E38
:105FF000046F000E056F010E066F000E076FDAECDE
:1060000036F047EC37F02AC182F40401300E8227C3
:106010004DEC0FF02BC182F40401300E82274DECC1
:106020000FF02CC182F40401300E82274DEC0FF0EA
:106030002DC182F40401300E82274DEC0FF02EC1E9
:1060400082F40401300E82274DEC0FF02FC182F450
:106050000401300E82274DEC0FF030C182F40401B0
:10606000300E82274DEC0FF031C182F40401300E66
:1060700082274DEC0FF004012E0E826F4DEC0FF0D5
:1060800032C182F40401300E82274DEC0FF033C18F
:1060900082F40401300E82274DEC0FF004016D0EE6
:1060A000826F4DEC0FF01200120EC5EC0BF0E8CF32
:1060B00000F1130EC5EC0BF0E8CF01F1140EC5ECA6
:1060C0000BF0E8CF02F1150EC5EC0BF0E8CF03F1B1
:1060D00001010A0E046F000E056F000E066F000E20
:1060E000076FBAEC36F0000E046F120E056F000E4B
:1060F000066F000E076FDAEC36F047EC37F02AC176
:1061000082F40401300E82274DEC0FF02BC182F493
:106110000401300E82274DEC0FF02CC182F40401F3
:10612000300E82274DEC0FF02DC182F40401300EA9
:1061300082274DEC0FF02EC182F40401300E82272D
:106140004DEC0FF02FC182F40401300E82274DEC8C
:106150000FF030C182F40401300E82274DEC0FF0B5
:1061600004012E0E826F4DEC0FF031C182F4040158
:10617000300E82274DEC0FF032C182F40401300E54
:1061800082274DEC0FF033C182F40401300E8227D8
:106190004DEC0FF00401730E826F4DEC0FF0120006
:1061A0000A0EC5EC0BF0E8CF00F10B0EC5EC0BF0BE
:1061B000E8CF01F10C0EC5EC0BF0E8CF02F10D0EAB
:1061C000C5EC0BF0E8CF03F105EF31F0060EC5EC9E
:1061D0000BF0E8CF00F1070EC5EC0BF0E8CF01F1B2
:1061E000080EC5EC0BF0E8CF02F1090EC5EC0BF080
:1061F000E8CF03F105EF31F00101A4EC37F007849B
:1062000057C100F158C101F107940101E80E046F74
:10621000800E056F000E066F000E076FBAEC36F0A9
:10622000000E046F040E056F000E066F000E076F60
:10623000DAEC36F0880E046F130E056F000E066F51
:10624000000E076FA9EC36F00A0E046F000E056F02
:10625000000E066F000E076FDAEC36F047EC37F0F1
:106260000101296739EF31F00401200E826F3CEF04
:1062700031F004012D0E826F4DEC0FF030C182F42D
:106280000401300E82274DEC0FF031C182F404017D
:10629000300E82274DEC0FF032C182F40401300E33
:1062A00082274DEC0FF004012E0E826F4DEC0FF0A3
:1062B00033C182F40401300E82274DEC0FF004014B
:1062C000430E826F4DEC0FF0120087C32AF188C392
:1062D0002BF189C32CF18AC32DF18BC32EF18CC312
:1062E0002FF18DC330F18EC331F190C332F191C3E0
:1062F00033F10101296BF2EC37F069EC37F0010161
:10630000000E046F000E056F010E066F000E076F82
:10631000BAEC36F00E0E0C6E00C10BF0AEEC0BF0CA
:106320000F0E0C6E01C10BF0AEEC0BF0100E0C6EEC
:1063300002C10BF0AEEC0BF0110E0C6E03C10BF0B2
:10634000AEEC0BF004017A0E826F4DEC0FF00401FD
:106350002C0E826F4DEC0FF00401350E826F4DEC68
:106360000FF004012C0E826F4DEC0FF0E1EC2FF0DA
:1063700075EF2AF087C32AF188C32BF189C32CF16A
:106380008AC32DF18BC32EF18CC32FF18DC330F155
:106390008EC331F190C332F191C333F10101296B06
:1063A000F2EC37F069EC37F0880E046F130E056FCE
:1063B000000E066F000E076FAEEC36F0000E046F95
:1063C000040E056F000E066F000E076FBAEC36F074
:1063D0000101E80E046F800E056F000E066F000EBF
:1063E000076FDAEC36F00A0E0C6E00C10BF0AEEC63
:1063F0000BF00B0E0C6E01C10BF0AEEC0BF00C0EA3
:106400000C6E02C10BF0AEEC0BF00D0E0C6E03C166
:106410000BF0AEEC0BF004017A0E826F4DEC0FF036
:1064200004012C0E826F4DEC0FF00401360E826FCA
:106430004DEC0FF004012C0E826F4DEC0FF0D0EC00
:1064400030F075EF2AF087C32AF188C32BF189C396
:106450002CF18AC32DF18BC32EF18CC32FF18DC388
:1064600030F18FC331F190C332F191C333F10101A7
:10647000F2EC37F069EC37F0000E046F120E056F86
:10648000000E066F000E076FBAEC36F001010A0E1F
:10649000046F000E056F000E066F000E076FDAEC3A
:1064A00036F0120E0C6E00C10BF0AEEC0BF0130EBA
:1064B0000C6E01C10BF0AEEC0BF0140E0C6E02C1B1
:1064C0000BF0AEEC0BF0150E0C6E03C10BF0AEEC46
:1064D0000BF004017A0E826F4DEC0FF004012C0ECC
:1064E000826F4DEC0FF00401370E826F4DEC0FF010
:1064F00004012C0E826F4DEC0FF054EC30F075EF70
:106500002AF087C32AF188C32BF189C32CF18AC3EF
:106510002DF18BC32EF18CC32FF18DC330F18EC3BF
:1065200031F190C332F191C333F10101296BF2ECE7
:1065300037F069EC37F0880E046F130E056F000E0C
:10654000066F000E076FAEEC36F0000E046F040EFF
:10655000056F000E066F000E076FBAEC36F00101F2
:10656000E80E046F800E056F000E066F000E076FB9
:10657000DAEC36F0060E0C6E00C10BF0AEEC0BF050
:10658000070E0C6E01C10BF0AEEC0BF0080E0C6E9A
:1065900002C10BF0AEEC0BF0090E0C6E03C10BF058
:1065A000AEEC0BF004017A0E826F4DEC0FF004019B
:1065B0002C0E826F4DEC0FF00401380E826F4DEC03
:1065C0000FF004012C0E826F4DEC0FF0E6EC30F072
:1065D00075EF2AF007A85DEF33F00101800E006F20
:1065E0001A0E016F060E026F000E036F4BC104F10D
:1065F0004CC105F14DC106F14EC107F1A9EC36F0D1
:1066000003BFA3EF33F004EC35F04BC100F14CC1F4
:1066100001F14DC102F14EC103F10782B6EC35F034
:1066200018C104F119C105F11AC106F11BC107F126
:10663000F80E006FCD0E016F660E026F030E036F32
:10664000A9EC36F00E0E0C6E00C10BF0AEEC0BF0A8
:106650000F0E0C6E01C10BF0AEEC0BF0100E0C6EB9
:1066600002C10BF0AEEC0BF0110E0C6E03C10BF07F
:10667000AEEC0BF007840101A4EC37F057C100F138
:1066800058C101F107940A0E0C6E00C10BF0AEEC7C
:106690000BF00B0E0C6E01C10BF0AEEC0BF00C0E00
:1066A0000C6E02C10BF0AEEC0BF00D0E0C6E03C1C4
:1066B0000BF0AEEC0BF0A3EF33F007AAA3EF33F02F
:1066C00007840101A4EC37F057C100F158C101F172
:1066D0000794060E0C6E00C10BF0AEEC0BF0070E2B
:1066E0000C6E01C10BF0AEEC0BF0080E0C6E02C18B
:1066F0000BF0AEEC0BF0090E0C6E03C10BF0AEEC20
:106700000BF0078462C100F163C101F164C102F1C1
:1067100065C103F10794120E0C6E00C10BF0AEECD4
:106720000BF0130E0C6E01C10BF0AEEC0BF0140E5F
:106730000C6E02C10BF0AEEC0BF0150E0C6E03C12B
:106740000BF0AEEC0BF00798079A04018051811909
:106750007F0B0DE09EA8FED714EE00F081517F0B59
:10676000E126E750812B0F01AD6EA5EF33F0050157
:106770002F51010A13E081AADFEF33F005012F51F9
:10678000000A0AE00FB8CEEF33F005013067CEEF14
:1067900033F00FB8CEEF33F07FEF41F081B8DFEF89
:1067A00033F0F3EC39F0DFEF33F0602FDFEF33F04D
:1067B0005FC560F50501010E306F3C0E316F8FEF44
:1067C0000EF006013251385D3351D8A0010F395D0A
:1067D000800BD8A4F0EF33F032C638F633C639F662
:1067E000120006013251365D3351D8A0010F375DDA
:1067F000800BD8B400EF34F032C636F633C637F625
:10680000120007841AC632F61BC633F61CC638F6C9
:106810001DC639F6E1EC33F01EC632F61FC633F65C
:10682000E1EC33F020C632F621C633F6E1EC33F06A
:106830001AC632F61BC633F61CC636F61DC637F628
:10684000F1EC33F01EC632F61FC633F6F1EC33F02E
:1068500020C632F621C633F6F1EC33F03851365FFC
:106860003951D8A03929375FA4EC37F036C600F18A
:1068700037C601F1B0EC37F000C13AF601C13BF682
:1068800022C632F623C633F624C638F625C639F6B4
:10689000E1EC33F026C632F627C633F6E1EC33F0EE
:1068A00028C632F629C633F6E1EC33F022C632F6BA
:1068B00023C633F624C636F625C637F6F1EC33F098
:1068C00026C632F627C633F6F1EC33F028C632F688
:1068D00029C633F6F1EC33F03851365F3951D8A080
:1068E0003929375FA4EC37F036C600F137C601F11D
:1068F000B0EC37F000C13CF601C13DF62AC632F6D5
:106900002BC633F62CC638F62DC639F6E1EC33F03B
:106910002EC632F62FC633F6E1EC33F030C632F62F
:1069200031C633F6E1EC33F02AC632F62BC633F625
:106930002CC636F62DC637F6F1EC33F02EC632F6FD
:106940002FC633F6F1EC33F030C632F631C633F6EB
:10695000F1EC33F03851365F3951D8A03929375F1F
:10696000A4EC37F036C600F137C601F1B0EC37F0D1
:1069700000C13EF601C13FF63AC632F63BC633F6D9
:106980003CC636F63DC637F6F1EC33F03EC632F67D
:106990003FC633F6F1EC33F00794120018C100F152
:1069A00019C101F11AC102F11BC103F1000E046FFC
:1069B000000E056F010E066F000E076FDAEC36F061
:1069C00029A1F9EF34F02051D8B4F9EF34F018C10F
:1069D00000F119C101F11AC102F11BC103F1000E4E
:1069E000046F000E056F0A0E066F000E076FDAECDB
:1069F00036F0120001010451001305510113065134
:106A000002130751031312000101186B196B1A6B63
:106A10001B6B12002AC182F40401300E82274DEC58
:106A20000FF02BC182F40401300E82274DEC0FF0E1
:106A30002CC182F40401300E82274DEC0FF02DC1E1
:106A400082F40401300E82274DEC0FF02EC182F447
:106A50000401300E82274DEC0FF02FC182F40401A7
:106A6000300E82274DEC0FF030C182F40401300E5D
:106A700082274DEC0FF031C182F40401300E8227E1
:106A80004DEC0FF032C182F40401300E82274DEC40
:106A90000FF033C182F40401300E82274DEC0FF069
:106AA00012002FC182F40401300E82274DEC0FF04A
:106AB00030C182F40401300E82274DEC0FF031C159
:106AC00082F40401300E82274DEC0FF032C182F4C3
:106AD0000401300E82274DEC0FF033C182F4040123
:106AE000300E82274DEC0FF01200060E1E6E060EC1
:106AF0001F6E060E206E1E2E7BEF35F01F2E7BEFD5
:106B000035F0202E7BEF35F08B84020E1E6E020EC8
:106B10001F6E020E206E1E2E8BEF35F01F2E8BEF98
:106B200035F0202E8BEF35F08B941200FF0E1F6E88
:106B30001FC020F0030E1E6E8B841E2E9CEF35F0BE
:106B4000030E1E6E202E9CEF35F08B941FC020F09C
:106B5000030E1E6E1E2EAAEF35F0030E1E6E203E93
:106B6000AAEF35F01F2E98EF35F012000101005307
:106B700005E1015303E1025301E1002B79EC36F00A
:106B8000A4EC37F03951006F3A51016F420E046F97
:106B90004B0E056F000E066F000E076FBAEC36F055
:106BA00000C104F101C105F102C106F103C107F101
:106BB00018C100F119C101F11AC102F11BC103F1A1
:106BC00007B2E7EF35F0AEEC36F0E9EF35F0A9ECBF
:106BD00036F000C118F101C119F102C11AF103C167
:106BE0001BF11200A4EC37F059C100F15AC101F1B8
:106BF000060EC5EC0BF0E8CF04F1070EC5EC0BF068
:106C0000E8CF05F1080EC5EC0BF0E8CF06F1090E50
:106C1000C5EC0BF0E8CF07F1A9EC36F000C124F188
:106C200001C125F102C126F103C127F1290E046F2C
:106C3000000E056F000E066F000E076FBAEC36F0FF
:106C4000EE0E046F430E056F000E066F000E076F09
:106C5000AEEC36F024C104F125C105F126C106F1E0
:106C600027C107F1BAEC36F000C11CF101C11DF1DA
:106C700002C11EF103C11FF1120EC5EC0BF0E8CFEB
:106C800004F1130EC5EC0BF0E8CF05F1140EC5ECC2
:106C90000BF0E8CF06F1150EC5EC0BF0E8CF07F1CD
:106CA0000D0E006F000E016F000E026F000E036FDD
:106CB000BAEC36F0180E046F000E056F000E066F6A
:106CC000000E076FDAEC36F01CC104F11DC105F1AE
:106CD0001EC106F11FC107F1AEEC36F06A0E046F5B
:106CE0002A0E056F000E066F000E076FA9EC36F036
:106CF0001200BF0EFA6E200E3A6F396BD890003733
:106D0000013702370337D8B08AEF36F03A2F7FEFDA
:106D100036F039073A070353D8B412000331070B92
:106D200080093F6F03390F0B010F396F80EC5FF063
:106D3000406F390580EC5FF0405D405F396B3F3359
:106D4000D8B0392739333FA99FEF36F04051392762
:106D500012000101C9EC37F0D8B012000101035153
:106D60000719346F8CEC37F0D8900751031934AF02
:106D7000800F12000101346BB0EC37F0D8A0C6ECE4
:106D800037F0D8B012009BEC37F0A4EC37F01F0EB0
:106D9000366FDCEC37F00B35D8B08CEC37F0D8A080
:106DA0000335D8B01200362FC9EF36F034B1B3EC4A
:106DB00037F012000101346B04510511061107115F
:106DC0000008D8A0B0EC37F0D8A0C6EC37F0D8B0A7
:106DD0001200086B096B0A6B0B6BDCEC37F01F0EB3
:106DE000366FDCEC37F007510B5DD8A404EF37F0B9
:106DF00006510A5DD8A404EF37F00551095DD8A407
:106E000004EF37F00451085DD8A017EF37F00451B4
:106E1000085F0551D8A0053D095F0651D8A0063D81
:106E20000A5F0751D8A0073D0B5FD8900081362F2D
:106E3000F1EF36F034B1B3EC37F0346BB0EC37F03F
:106E4000D890E0EC37F007510B5DD8A434EF37F061
:106E500006510A5DD8A434EF37F00551095DD8A476
:106E600034EF37F00451085DD8A043EF37F0003F0E
:106E700043EF37F0013F43EF37F0023F43EF37F086
:106E8000032BD8B4120034B1B3EC37F01200010177
:106E9000346BB0EC37F0D8B01200E5EC37F0200ED0
:106EA000366F003701370237033711EE33F00A0E21
:106EB000376FE7360A0EE75CD8B0E76EE552372F3A
:106EC00059EF37F0362F51EF37F034B12981D89090
:106ED000120001010A0E346F200E366F11EE29F0F8
:106EE0003451376F0A0ED890E652D8B0E726E73211
:106EF000372F74EF37F00333023301330033362F6B
:106F00006EEF37F0E750FF0FD8A00335D8B012006E
:106F100029B1B3EC37F01200045100270551D8B065
:106F2000053D01270651D8B0063D02270751D8B0CC
:106F3000073D032712000051086F0151096F0251EC
:106F40000A6F03510B6F12000101006B016B026BA2
:106F5000036B12000101046B056B066B076B1200DB
:106F60000335D8A012000351800B001F011F021F20
:106F7000031F003FC3EF37F0013FC3EF37F0023F7D
:106F8000C3EF37F0032B342B032512000735D8A0AD
:106F900012000751800B041F051F061F071F043F27
:106FA000D9EF37F0053FD9EF37F0063FD9EF37F08B
:106FB000072B342B07251200003701370237033720
:106FC000083709370A370B3712000101296B2A6B82
:106FD0002B6B2C6B2D6B2E6B2F6B306B316B326BE5
:106FE000336B120001012A510F0B2A6F2B510F0B2B
:106FF0002B6F2C510F0B2C6F2D510F0B2D6F2E5112
:107000000F0B2E6F2F510F0B2F6F30510F0B306F57
:1070100031510F0B316F32510F0B326F33510F0B58
:10702000336F1200899C000EC76E200EC66E9E96AE
:10703000C69EC50EC96EFF0E9EB602D0E82EFCD7C6
:107040009E96C69E000EC96EFF0E9EB602D0E82E1A
:10705000FCD7C9CF00F69E96C69E000EC96EFF0EE5
:107060009EB602D0E82EFCD7C9CF01F6898C12005B
:10707000000EC76E200EC66E899C9E96C69EC80ED8
:10708000C96EFF0E9EB602D0E82EFCD79E96C69E15
:10709000000EC96EFF0E9EB602D0E82EFCD7C9CFF7
:1070A00002F69E96C69E000EC96EFF0E9EB602D0D8
:1070B000E82EFCD7C9CF03F69E96C69E000EC96E79
:1070C000FF0E9EB602D0E82EFCD7C9CF0AF69E96D8
:1070D000C69E000EC96EFF0E9EB602D0E82EFCD7EB
:1070E000C9CF0BF69E96C69E000EC96EFF0E9EB6C9
:1070F00002D0E82EFCD7C9CF12F69E96C69E000E8F
:10710000C96EFF0E9EB602D0E82EFCD7C9CF13F68B
:10711000898C1200000EC76E200EC66E899C9E964A
:10712000C69EE80EC96EFF0E9EB602D0E82EFCD7B2
:107130009E96C69E000EC96EFF0E9EB602D0E82E29
:10714000FCD7C9CF1AF69E96C69E000EC96EFF0EDA
:107150009EB602D0E82EFCD7C9CF1BF69E96C69EDF
:10716000000EC96EFF0E9EB602D0E82EFCD7C9CF26
:1071700022F69E96C69E000EC96EFF0E9EB602D0E7
:10718000E82EFCD7C9CF23F69E96C69E000EC96E88
:10719000FF0E9EB602D0E82EFCD7C9CF2AF69E96E7
:1071A000C69E000EC96EFF0E9EB602D0E82EFCD71A
:1071B000C9CF2BF6898C1200000EC76E200EC66E4A
:1071C000899C9E96C69E240EC96EFF0E9EB602D066
:1071D000E82EFCD79E96C69EE40EC96EFF0E9EB6A4
:1071E00002D0E82EFCD7898C899C9E96C69E200EE4
:1071F000C96EFF0E9EB602D0E82EFCD79E96C69EA4
:107200005F0EC96EFF0E9EB602D0E82EFCD7898CA9
:10721000899C9E96C69E210EC96EFF0E9EB602D018
:10722000E82EFCD79E96C69EC00EC96EFF0E9EB677
:1072300002D0E82EFCD7898C899C9E96C69E260E8D
:10724000C96EFF0E9EB602D0E82EFCD79E96C69E53
:10725000000EC96EFF0E9EB602D0E82EFCD7898CB8
:10726000120010A806D08994000EC76E220EC66EBA
:1072700005D08984000EC76E220EC66E050EE82E5C
:10728000FED7120010A802D0898401D08994050E7F
:10729000E82EFED7120031EC39F09E96C69E000E05
:1072A000C96EFF0E9EB602D0E82EFCD79E96C69EF3
:1072B000000EC96EFF0E9EB602D0E82EFCD7C9CFD5
:1072C000AFF59E96C69E000EC96EFF0E9EB602D00A
:1072D000E82EFCD7C9CFB0F59E96C69E000EC96EAB
:1072E000FF0E9EB602D0E82EFCD7C9CFB1F59E9610
:1072F000C69E000EC96EFF0E9EB602D0E82EFCD7C9
:10730000C9CFB2F59E96C69E000EC96EFF0E9EB600
:1073100002D0E82EFCD7C9CFB3F59E96C69E000ECC
:10732000C96EFF0E9EB602D0E82EFCD7C9CFB4F5C9
:107330009E96C69E000EC96EFF0E9EB602D0E82E27
:10734000FCD7C9CFB5F542EC39F0120031EC39F079
:107350009E96C69E800EC96EFF0E9EB602D0E82E87
:10736000FCD79E96C69EAFC5C9FFFF0E9EB602D043
:10737000E82EFCD79E96C69EB0C5C9FFFF0E9EB6EE
:1073800002D0E82EFCD79E96C69EB1C5C9FFFF0E5F
:107390009EB602D0E82EFCD79E96C69EB2C5C9FF07
:1073A000FF0E9EB602D0E82EFCD79E96C69EB3C5B1
:1073B000C9FFFF0E9EB602D0E82EFCD79E96C69E51
:1073C000B4C5C9FFFF0E9EB602D0E82EFCD79E962C
:1073D000C69EB5C5C9FFFF0E9EB602D0E82EFCD7EB
:1073E00042EC39F0120031EC39F09E96C69E070E41
:1073F000C96EFF0E9EB602D0E82EFCD79E96C69EA2
:10740000000EC96EFF0E9EB602D0E82EFCD7C9CF83
:10741000AFF59E96C69E000EC96EFF0E9EB602D0B8
:10742000E82EFCD7C9CFB0F59E96C69E000EC96E59
:10743000FF0E9EB602D0E82EFCD7C9CFB1F59E96BE
:10744000C69E000EC96EFF0E9EB602D0E82EFCD777
:10745000C9CFB2F542EC39F031EC39F09E96C69EB8
:1074600022C0C9FFFF0E9EB602D0E82EFCD79E9622
:10747000C69E000EC96EFF0E9EB602D0E82EFCD747
:10748000C9CFB6F542EC39F0120031EC39F09E96D6
:10749000C69E870EC96EFF0E9EB602D0E82EFCD7A0
:1074A0009E96C69EAFC5C9FFFF0E9EB602D0E82EBF
:1074B000FCD79E96C69EB0C5C9FFFF0E9EB602D0F1
:1074C000E82EFCD79E96C69EB1C5C9FFFF0E9EB69C
:1074D00002D0E82EFCD79E96C69EB2C5C9FFFF0E0D
:1074E0009EB602D0E82EFCD742EC39F031EC39F0F0
:1074F0009E96C69E23C0C9FFFF0E9EB602D0E82E00
:10750000FCD79E96C69EB6C5C9FFFF0E9EB602D09A
:10751000E82EFCD742EC39F0120031EC39F09E969F
:10752000C69E870EC96EFF0E9EB602D0E82EFCD70F
:107530009E96C69E000EC96EFF0E9EB602D0E82E25
:10754000FCD79E96C69E800EC96EFF0E9EB602D0D8
:10755000E82EFCD79E96C69E800EC96EFF0E9EB684
:1075600002D0E82EFCD79E96C69E800EC96EFF0EF6
:107570009EB602D0E82EFCD742EC39F0120031EC76
:1075800039F09E96C69E870EC96EFF0E9EB602D03B
:10759000E82EFCD79E96C69E000EC96EFF0E9EB6C4
:1075A00002D0E82EFCD79E96C69E000EC96EFF0E36
:1075B0009EB602D0E82EFCD79E96C69E800EC96E5F
:1075C000FF0E9EB602D0E82EFCD79E96C69E800E79
:1075D000C96EFF0E9EB602D0E82EFCD742EC39F001
:1075E000120010A817D031EC39F09E96C69E8F0E6F
:1075F000C96EFF0E9EB602D0E82EFCD79E96C69EA0
:10760000000EC96EFF0E9EB602D0E82EFCD742ECEB
:1076100039F01200F3EC39F0120010A82DD031EC43
:1076200039F09E96C69E23C0C9FFFF0E9EB602D0BB
:10763000E82EFCD79E96C69E450EC96EFF0E9EB6DE
:1076400002D0E82EFCD742EC39F031EC39F09E96AE
:10765000C69E8F0EC96EFF0E9EB602D0E82EFCD7D6
:107660009E96C69E000EC96EFF0E9EB602D0E82EF4
:10767000FCD742EC39F0120031EC39F09E96C69EF0
:1076800023C0C9FFFF0E9EB602D0E82EFCD79E96FF
:10769000C69E010EC96EFF0E9EB602D0E82EFCD724
:1076A00042EC39F031EC39F09E96C69E910EC96ECF
:1076B000FF0E9EB602D0E82EFCD79E96C69EA50E63
:1076C000C96EFF0E9EB602D0E82EFCD742EC39F010
:1076D000120031EC39F09E96C69E23C0C9FFFF0E02
:1076E0009EB602D0E82EFCD79E96C69E810EC96E2D
:1076F000FF0E9EB602D0E82EFCD742EC39F0120005
:1077000031EC39F09E96C69E23C0C9FFFF0E9EB68F
:1077100002D0E82EFCD79E96C69E010EC96EFF0EC3
:107720009EB602D0E82EFCD742EC39F0120031ECC4
:1077300039F09E96C69E910EC96EFF0E9EB602D07F
:10774000E82EFCD79E96C69EA50EC96EFF0E9EB66D
:1077500002D0E82EFCD742EC39F0120031EC39F0BF
:107760009E96C69E910EC96EFF0E9EB602D0E82E62
:10777000FCD79E96C69E000EC96EFF0E9EB602D026
:10778000E82EFCD742EC39F012000501256B266B80
:10779000276B286B899A400EC76E200EC66E9E9688
:1077A000C69E030EC96EFF0E9EB602D0E82EFCD711
:1077B0009E96C69E27C5C9FFFF0E9EB602D0E82E34
:1077C000FCD79E96C69E26C5C9FFFF0E9EB602D068
:1077D000E82EFCD79E96C69E25C5C9FFFF0E9EB615
:1077E00002D0E82EFCD79E96C69EC952FF0E9EB6CA
:1077F00002D0E82EFCD7898A0F01C950FF0A01E1A7
:10780000120005012E51130A05E005012E51170A39
:107810000CE012000501E00E256FFF0E266F0F0E23
:10782000276F000E286F1EEF3CF00501E00E256F5C
:10783000FF0E266FFF0E276F000E286F899A400EED
:10784000C76E200EC66E9E96C69E030EC96EFF0EB4
:107850009EB602D0E82EFCD79E96C69E27C5C9FFCD
:10786000FF0E9EB602D0E82EFCD79E96C69E26C579
:10787000C9FFFF0E9EB602D0E82EFCD79E96C69E8C
:1078800025C5C9FFFF0E9EB602D0E82EFCD79E96F6
:10789000C69EC952FF0E9EB602D0E82EFCD7898A3A
:1078A0000F01C950FF0A1DE005012E51130A05E022
:1078B00005012E51170A0BE012000501000E256F7D
:1078C000000E266F100E276F000E286F12000501A4
:1078D000000E256F000E266F000E276F010E286F19
:1078E00012000501256B266B276B286B05012E51B5
:1078F000130A05E005012E51170A0CE012000501DC
:10790000000E216F000E226F080E236F000E246FF1
:1079100093EF3CF00501000E216F000E226F800EE8
:10792000236F000E246F21C500F122C501F123C58C
:1079300002F124C503F125C504F126C505F127C5CB
:1079400006F128C507F1FAEC34F000C125F501C1B4
:1079500026F502C127F503C128F5899A400EC76EA6
:10796000200EC66E9E96C69E030EC96EFF0E9EB674
:1079700002D0E82EFCD79E96C69E27C5C9FFFF0EF3
:107980009EB602D0E82EFCD79E96C69E26C5C9FF9D
:10799000FF0E9EB602D0E82EFCD79E96C69E25C549
:1079A000C9FFFF0E9EB602D0E82EFCD79E96C69E5B
:1079B000C952FF0E9EB602D0E82EFCD7898AC95064
:1079C000FF0A08E104C125F505C126F506C127F522
:1079D00007C128F5D89005012433233322332133FE
:1079E0002151E00B216F2167FDEF3CF02267FDEF95
:1079F0003CF02367FDEF3CF0246793EF3CF005017A
:107A0000200E2527E86A2623E86A2723E86A282328
:107A10001200E86A05012E51130A06E005012E51F5
:107A2000170A0BE0020E120005012851000A03E1BB
:107A30002751F00B07E0010E120005012851000A42
:107A400001E0010E120029C500F12AC501F12BC584
:107A500002F12CC503F125C504F126C505F127C5A2
:107A600006F128C507F1A9EC36F003BF120009ECB6
:107A70003DF0D8A49BEF3DF0899A400EC76E200ED2
:107A8000C66E9E96C69E060EC96EFF0E9EB602D0AC
:107A9000E82EFCD7898A899A9E96C69E020EC96EE8
:107AA000FF0E9EB602D0E82EFCD79E96C69E27C536
:107AB000C9FFFF0E9EB602D0E82EFCD79E96C69E4A
:107AC00026C5C9FFFF0E9EB602D0E82EFCD79E96B3
:107AD000C69E25C5C9FFFF0E9EB602D0E82EFCD774
:107AE0009E96C69E000EC96EFF0E9EB602D0E82E70
:107AF000FCD7898A899A9E96C69E050EC96EFF0E8E
:107B00009EB602D0E82EFCD79E96C69EC952FF0EA6
:107B10009EB602D0E82EFCD7C9B084EF3DF0898A2A
:107B20000501200E2527E86A2623E86A2723E86A4C
:107B3000282323EF3DF01200899A400EC76E200ED5
:107B4000C66E9E96C69E060EC96EFF0E9EB602D0EB
:107B5000E82EFCD7898A899A9E96C69EC70EC96E62
:107B6000FF0E9EB602D0E82EFCD7898A0501256B50
:107B7000266B276B286B1200899A400EC76E200E69
:107B8000C66E9E96C69E050EC96EFF0E9EB602D0AC
:107B9000E82EFCD79E96C69EC952FF0E9EB602D016
:107BA000E82EFCD7C9CF37F5898A1200899A400E92
:107BB000C76E200EC66E9E96C69EB90EC96EFF0E8B
:107BC0009EB602D0E82EFCD7898A1200899A400E10
:107BD000C76E200EC66E9E96C69EAB0EC96EFF0E79
:107BE0009EB602D0E82EFCD7898AFF0EE82EFED77B
:107BF000120009EC3DF0D8A41200899A400EC76E1D
:107C0000200EC66E9E96C69E030EC96EFF0E9EB6D1
:107C100002D0E82EFCD79E96C69E27C5C9FFFF0E50
:107C20009EB602D0E82EFCD79E96C69E26C5C9FFFA
:107C3000FF0E9EB602D0E82EFCD79E96C69E25C5A6
:107C4000C9FFFF0E9EB602D0E82EFCD79E96C69EB8
:107C5000C952FF0E9EB602D0E82EFCD7898A0F01CA
:107C6000C950FF0AD8A4F2EF40F00501FE0E376FAD
:107C700030A037994BEC39F0AFC538F5B0C539F5C0
:107C8000B1C53AF5B2C53BF5B3C53CF5B4C53DF554
:107C9000B5C53EF50784B6C166F1B7C167F1B8C195
:107CA00068F1B9C169F14BC14FF14CC150F14DC1FF
:107CB00051F14EC152F157C159F158C15AF19FECDF
:107CC0002AF000C13FF501C140F502C141F503C1F1
:107CD00042F50501616774EF3EF0626774EF3EF0B4
:107CE000636774EF3EF0646778EF3EF085EF3EF037
:107CF00061C504F162C505F163C506F164C507F10C
:107D0000A9EC36F003BFF2EF40F059C143F55AC178
:107D100044F5B9C545F5BAC546F501EC34F036C6AB
:107D200049F537C64AF5060140679EEF3EF04167C8
:107D30009EEF3EF042679EEF3EF04367A2EF3EF0BB
:107D4000B3EF3EF0A4EC37F0AAEC37F036C600F102
:107D500037C601F140C604F141C605F1A9EC36F081
:107D600003AFF2EF40F00101036B026B1AC600F1A2
:107D70001BC601F101AFC1EF3EF0FF0E026FFF0E17
:107D8000036F0101076B066B1CC604F11DC605F1EC
:107D900005AFCFEF3EF0FF0E066FFF0E076FAEECA4
:107DA00036F00101076B066B1EC604F11FC605F114
:107DB00005AFDFEF3EF0FF0E066FFF0E076FAEEC74
:107DC00036F00101076B066B20C604F121C605F1F0
:107DD00005AFEFEF3EF0FF0E066FFF0E076FAEEC44
:107DE00036F0D89001010333023301330033D890C9
:107DF0000101033302330133003300C14BF501C1EC
:107E00004CF50101036B026B22C600F123C601F1A0
:107E100001AF0FEF3FF0FF0E026FFF0E036F010186
:107E2000076B066B24C604F125C605F105AF1DEFEF
:107E30003FF0FF0E066FFF0E076FAEEC36F001014C
:107E4000076B066B26C604F127C605F105AF2DEFBB
:107E50003FF0FF0E066FFF0E076FAEEC36F001012C
:107E6000076B066B28C604F129C605F105AF3DEF87
:107E70003FF0FF0E066FFF0E076FAEEC36F0D890A6
:107E800001010333023301330033D890010103337E
:107E900002330133003300C14DF501C14EF501013C
:107EA000036B026B2AC600F12BC601F101AF5DEF37
:107EB0003FF0FF0E026FFF0E036F0101076B066BB1
:107EC0002CC604F12DC605F105AF6BEF3FF0FF0E98
:107ED000066FFF0E076FAEEC36F00101076B066B05
:107EE0002EC604F12FC605F105AF7BEF3FF0FF0E64
:107EF000066FFF0E076FAEEC36F00101076B066BE5
:107F000030C604F131C605F105AF8BEF3FF0FF0E2F
:107F1000066FFF0E076FAEEC36F0D8900101033309
:107F2000023301330033D8900101033302330133AC
:107F3000003300C14FF501C150F50101036B026B25
:107F400002C600F103C601F101AFABEF3FF0FF0E37
:107F5000026FFF0E036F0101076B066B04C604F18D
:107F600005C605F105AFB9EF3FF0FF0E066FFF0E36
:107F7000076FAEEC36F00101076B066B06C604F125
:107F800007C605F105AFC9EF3FF0FF0E066FFF0E04
:107F9000076FAEEC36F00101076B066B08C604F103
:107FA00009C605F105AFD9EF3FF0FF0E066FFF0ED2
:107FB000076FAEEC36F0D890010103330233013382
:107FC0000033D8900101033302330133003300C181
:107FD00051F501C152F50101036B026B0AC600F1B4
:107FE0000BC601F101AFF9EF3FF0FF0E026FFF0E7C
:107FF000036F0101076B066B0CC604F10DC605F19A
:1080000005AF07EF40F0FF0E066FFF0E076FAEECF7
:1080100036F00101076B066B0EC604F10FC605F1C1
:1080200005AF17EF40F0FF0E066FFF0E076FAEECC7
:1080300036F00101076B066B10C604F111C605F19D
:1080400005AF27EF40F0FF0E066FFF0E076FAEEC97
:1080500036F0D89001010333023301330033D89056
:108060000101033302330133003300C153F501C171
:1080700054F50101036B026B12C600F113C601F146
:1080800001AF47EF40F0FF0E026FFF0E036F0101DB
:10809000076B066B14C604F115C605F105AF55EF65
:1080A00040F0FF0E066FFF0E076FAEEC36F00101D9
:1080B000076B066B16C604F117C605F105AF65EF31
:1080C00040F0FF0E066FFF0E076FAEEC36F00101B9
:1080D000076B066B18C604F119C605F105AF75EFFD
:1080E00040F0FF0E066FFF0E076FAEEC36F0D89033
:1080F00001010333023301330033D890010103330C
:1081000002330133003300C155F501C156F5079420
:108110000501210E326F899A400EC76E200EC66E81
:108120009E96C69E060EC96EFF0E9EB602D0E82E23
:10813000FCD7898A899A9E96C69E020EC96EFF0E4A
:108140009EB602D0E82EFCD79E96C69E27C5C9FFD4
:10815000FF0E9EB602D0E82EFCD79E96C69E26C580
:10816000C9FFFF0E9EB602D0E82EFCD79E96C69E93
:1081700025C5C9FFFF0E9EB602D0E82EFCD725EE1E
:1081800037F0322F02D0D0EF40F09E96C69EDECF61
:10819000C9FFFF0E9EB602D0E82EFCD7C1EF40F01B
:1081A000898A899A9E96C69E050EC96EFF0E9EB656
:1081B00002D0E82EFCD79E96C69EC952FF0E9EB6F0
:1081C00002D0E82EFCD7C9B0DBEF40F0898A050168
:1081D000200E2527E86A2623E86A2723E86A282351
:1081E00075EC35F0120021C500F122C501F123C55F
:1081F00002F124C503F1899A400EC76E200EC66EA7
:108200009E96C69E0B0EC96EFF0E9EB602D0E82E3D
:10821000FCD79E96C69E02C1C9FFFF0E9EB602D035
:10822000E82EFCD79E96C69E01C1C9FFFF0E9EB6E2
:1082300002D0E82EFCD79E96C69E00C1C9FFFF0E55
:108240009EB602D0E82EFCD79E96C69EC952FF0E5F
:108250009EB602D0E82EFCD725EE37F00501200EA1
:10826000326F9E96C69EC952FF0E9EB602D0E82E71
:10827000FCD7C9CFDEFF322F31EF41F0898A1200DF
:10828000899A400EC76E200EC66E9E96C69E900EB0
:10829000C96EFF0E9EB602D0E82EFCD79E96C69EF3
:1082A000000EC96EFF0E9EB602D0E82EFCD79E9639
:1082B000C69E000EC96EFF0E9EB602D0E82EFCD7F9
:1082C0009E96C69E000EC96EFF0E9EB602D0E82E88
:1082D000FCD79E96C69EC952FF0E9EB602D0E82ECF
:1082E000FCD7C9CF2DF59E96C69EC952FF0E9EB6ED
:1082F00002D0E82EFCD7C9CF2EF5898A120075EC82
:1083000035F0B9C5E8FFD70802E375EC35F0B9C51B
:10831000E8FFC80802E375EC35F0B9C5E8FFB90815
:1083200002E375EC35F0B9C5E8FFAA0802E375EC85
:1083300035F0B9C5E8FF9B0802E375EC35F0D6ECE3
:108340003DF0F29CF29E8B94C69AC290898C9482E6
:10835000948C720ED36ED3A4FED789968A90939094
:10836000F29AF2949D909E909D929E92F298F29233
:10837000F1EC3AF0FF0EE8CF00F0E82EFED7002E29
:10838000FCD7F290F286815081A8C9EF41F0F29EAD
:108390000300F296F290010E306E038096EC35F0F9
:0483A000FAEF0BF0F5
:10BF0000E844F926000C160C2B0C3F0C520C640C68
:10BF1000760C860C960CA50CB30CC10CCF0CDC0C6B
:06BF2000E80CF40C000C1B
:00000001FF
